:100000004D424E014D3448300502040001002200EB
:100010006000000000C000000000000000000000C0
:100020000000EEEE000000000000000000000000F4
:1000300001000502000000000000000000000000B8
:100040000200050100002D000000000000B40000C7
:10005000030005012D00300000B40000000C00007A
:10006000001C0020ED020000000000000000000065
:100070000000000000000000000000000000000080
:100080000000000000000000000000000000000070
:10009000000000000000000000000000B5010000AA
:1000A000E1010000FD010000B9010000CD010000E8
:1000B00000000000002934D00123002210B488423F
:1000C0002CD301242407A14204D2814202D2090187
:1000D0001B01F8E7E400A14204D2814202D24900A8
:1000E0005B00F8E7884201D3401A1A434C08A0424B
:1000F00002D3001B5C0822438C08A04202D3001BE1
:100100009C082243CC08A04202D3001BDC082243F7
:10011000002803D01B0901D00909E3E7101C10BC1B
:100120007047002801D00020C04307B4024802A154
:100130004018029003BDC046D90000000029F0D04D
:1001400003B5FFF7B9FF0EBC4243891A1847C046F2
:10015000002941D010B4041C4C40A44601230022C5
:10016000002900D54942002800D5404288422CD3BE
:1001700001242407A14204D2814202D209011B01B9
:10018000F8E7E400A14204D2814202D249005B00B8
:10019000F8E7884201D3401A1A434C08A04202D320
:1001A000001B5C0822438C08A04202D3001B9C0861
:1001B0002243CC08A04202D3001BDC0822430028C3
:1001C00003D01B0901D00909E3E7101C6446002C89
:1001D00000D5404210BC7047002806D003DB002049
:1001E000C043400801E08020000607B4024802A195
:1001F0004018029003BDC046190000000029EBD052
:1002000003B5FFF7A7FF0EBC4243891A1847C04643
:100210007047C046FEE70000034B01225A70A0233E
:100220000022DB051A707047800C0020034B01226E
:100230009A70A0230022DB059A707047800C002082
:1002400008B5044B01221A70034B0022DA7700F044
:10025000E9FE08BD800C00200800005038B580255C
:10026000ED052B79DBB2002B0CD130490B604B60D4
:100270002B89081C9BB28B608A680C30103106F009
:10028000E7FC47E0012B0DD1284BD968002941D06C
:100290005A68186982423DDA5A68501C58602B7AB5
:1002A0008B5437E0022B30D1204CE368002B2AD04E
:1002B000226821698A420CDA22689B5C1BBAEB60D7
:1002C000A3682068C01880B206F00CFD23680133D3
:1002D00017E0A2682368201C211CD2180C301031B2
:1002E00006F0B6FCE368002B0DD0A16822688A18DE
:1002F000A2601B781BBAEB60A06880B206F0F2FC2B
:100300000123236006E0EB6004E0032B02D1074BDE
:1003100000225A60C0468023DB0501221A70C046C5
:1003200002221A7000221A7038BDC0460C03002049
:1003300080230222DB05FF321A600421024AFF31CA
:10034000118000221A70704706000040F8B5A02303
:10035000DB059B68494A1F21DBB21160D12B0BD012
:10036000D02B01D80133DBB2A022D2059168FF2047
:10037000814319439160F1E70023414A41499A18AA
:100380008A4204D24049C95804331160F5E73F4B13
:100390003F4A191D043B934203D200221A600B1CF2
:1003A000F6E7EFF308823B4B191D043B9A4203D951
:1003B000394818600B1CF7E7FFF7BAFF3749384890
:1003C000053904F0EBF8374C374D01235B422371BC
:1003D0006371A371E3712B1C3C331A782B1C3D33E2
:1003E0001B7880B21B02134398423FD106F018FCE1
:1003F0002E4B2F4918882F4A88420BD06E7D1888C3
:100400002B7D36023343984204D113889BB223716B
:100410001B0A637113888B421BD0EE7DA87D138865
:1004200036023043834214D100200423013BDBB267
:10043000FF2B07D0204EEF18F65C3F79B742F5D17D
:100440000120F3E7002804D013889BB2A3711B0A94
:10045000E371637922791B0213438B4206D0E27960
:10046000A37912021A43124B9A4204D1134B02226F
:100470001A6062B6FEE701F021F9F7E728000050A4
:10048000000000200C030020389D00001003002015
:100490007C0C0020C80C0020CDCDCDCD00C00000CC
:1004A00000000000840C0020C0BF0000FEB300006C
:1004B000FFFF0000BEBF000000B4000000E100E04C
:1004C000014B18607047C0468C0C0020014B186827
:1004D0007047C0468C0C0020014B18607047C04626
:1004E000900C0020014B18687047C046900C00200B
:1004F000014B18687047C0460000002038B5134C07
:10050000256804F079FC6862256804F079FCA8622B
:10051000256804F079FC6861256804F079FCE861DD
:10052000256804F0C1FCA861256804F0D1FC084BE3
:1005300008491B68096828621878097C22684143C9
:1005400002331161E832136038BDC046000000205C
:10055000900C00208C0C002082B0F0B589B0109C6B
:10056000151C0F930693029407900E1C119C03F028
:1005700093FF47793A4B04978279964206D11B68DC
:100580000021DA69AB00D05A03910BE01A68354BB1
:1005900052691968731C896803964B43EB18013341
:1005A0009B00D05A0499714349194A00A418238822
:1005B000069E0193019F7318874203D8C61B029FB2
:1005C000BE521CE0029EB61805960027F65F013663
:1005D00010D01F787EB2B446013601DA013703E04D
:1005E0006646002E06DD013F1F7002235B4223801A
:1005F00001202FE0069F79180F78002F01D120806D
:100600000CE07FB27C1C05D1019E059F301A38801A
:10061000002002E0012F01D1FF2008701978039C0F
:10062000049E079F48B274437D19002805DC029E92
:10063000B25E013208D0002906D12A5700203E2A96
:1006400008DC0131197005E02A57002A01DD013963
:100650001970002009B0F0BC08BC02B01847C046B1
:1006600000000020F8020020F0B58BB000AF03F0CE
:1006700013FF06F083FB584C6E4623689D68DB68C9
:100680007D625A00111C0E319B00C9080E33C9004F
:10069000DB08DB00761AB546F61A6D46002168467F
:1006A000B546BD61FE6008F05DFD002004F0E2FC8F
:1006B0007E6A4A4A20681568B20052420368BA60EE
:1006C000321C5A439100F961B107711A79609107A0
:1006D000891A3A62013B32D344683E6A3219261CB9
:1006E0005E437618B400FE68920034197C61FC69A0
:1006F000A2420BD07C690426A418A4466C697642F9
:10070000A458B44466463460043AF0E7BE683A6AD6
:10071000A419FC617C6A7E68121B3A628919D9E7C8
:100720002F49F8697E23D2B25B4208704A708A7002
:10073000CB7001205223BA690B7106F017FA06F04C
:10074000EBF80B2845D1002004F094FC224B1968EB
:10075000224B08681C687B6AF86143439A003A623E
:100760009A07D21A3A617B61844666464A68013E1E
:10077000B446D5D3654655437E691A48B318121856
:100780005219BE6938695200B2182D18FE68AD00C2
:1007900075199B003D603E6AB3420ED03D68E81873
:1007A000656904380668E858301A0025565F8642A5
:1007B00000DA1080043B023AEDE7BD6876193E622C
:1007C0007D6A7E69761B7E617D683E6976193E6131
:1007D000CBE7BD460BB0F0BDF802002000000020C2
:1007E000B8030020FFFFFF7F08B502F0E9FA021E00
:1007F00005D10749A9230B7106F0B8F9FEE7054BAF
:100800001B6803CB03F05AFFFFF778FE08BDC04614
:10081000BF030020F8020020104B00221B6810B517
:10082000191C88310A601C1C01219C344942181C87
:100830002160A2600830083CE18222606283C267C6
:1008400090300160826008380183191CAC3102606D
:1008500020390A8404330A60DA6710BD00000020E2
:10086000F0B585B000AFB960386004F08FFD83004B
:100870000A33DB08DB00041C6846C01A854604F016
:100880008BFD63000833DB08DB006E46F11A8D46F2
:100890006D46281C7D6004F099FD4D4B1B68191CAA
:1008A00088310868632807DD0120002240420A6081
:1008B0004861CA61191DCA67191C883108681A1C69
:1008C000013008320860D16F63290CDD01204042FD
:1008D0008446181C002198306546D1678160056008
:1008E000191D0120C867D16F0131D1671A1C9432DC
:1008F000106801280BDD012040428446181C0021AD
:10090000AA30654611601E38C583418401601168B4
:1009100001311160191C90310868012809DD00229D
:1009200001200A608A8340421A1C08838C3201210C
:1009300011601A1C90321168013111600022101CE4
:10094000013C07D3A10071587D6840186100695AC5
:100950005218F5E7191CAA310024A4251E19AC462B
:10096000B444FE6066463668864201D26546286019
:10097000FD689C352E68864200D928608D88954296
:1009800000D28A800D88954200D90A80043C251C3B
:1009900002390835E1D11A1DD26F3E6892009A18CB
:1009A000111CA031983209681268BD688A1A328019
:1009B0001A1C8C321268BD4652009B181A1CAC32AD
:1009C000A83312881B88D31A2B8005B0F0BDC0460F
:1009D00000000020F0B5234F1D1C3B68161CDA6890
:1009E00085B0019192000021041C301C08F0BAFB74
:1009F0003B68281C1A690021920008F0B3FB019F94
:100A0000002F0CD0201C04F035FB174B301C1B684A
:100A1000291C5A69DB6906F0BBFA013FF0E7002C9C
:100A20000FD1114B1B685F699B69029304F0D2F9E7
:100A3000039004F0D9F90299031C039A381C06F0BC
:100A4000BBF9301C291C019A06F018FB002C06D1BA
:100A5000054B201C1D6804F033FCEC35286005B004
:100A6000F0BDC046F802002000000020F0B5274D80
:100A700087B02B680591DA6900219200039008F095
:100A800071FB06F087F904904478002C25D00420EF
:100A900004F0F0FA286842690292029B013B01933C
:100AA00019D383690199039E5943C91889007118A4
:100AB0000439013B0DD38668029F7E439E19059F32
:100AC0000136B600F2590E689446B44467460F608A
:100AD000EEE7019AE0E7013CD7E72F687D69013D29
:100AE00011D3BC69039A261C6E433619B6009619B9
:100AF000043E013CF3D3049B30685978FFF7DAFADF
:100B000000043060F4E707B0F0BDC046F8020020F2
:100B100030B5214D85B02B681A1CCC321178583A6B
:100B2000002904D1191CB0310978002901D0002115
:100B300011701478002C1DD0996F002001915A6B10
:100B400016490292DB6A01AA039303234B707C23AC
:100B50005B42CB7010230B7106F008F82B68002461
:100B60009A6FD96F8A4202DC01329A6710E09C6763
:100B700001240DE05A6BDB6A0949019202930920B6
:100B8000642301AA0B71039405F0F0FF2B689C67A6
:100B9000201C05B030BDC04600000020040100202C
:100BA0000B010020F0B58FB004AF7960BA617B61B2
:100BB000B86006F0EFF8934B69461B6838611C6813
:100BC000F96104346400221C0832D208D200881A69
:100BD0005A68854604325200131C0833DB08DB00D8
:100BE000C01A04AE854604AD281C002108F0BAFAEC
:100BF000221C301C002108F0B5FA834CB868236829
:100C00005A69191C9B690090301D0190281D0290A3
:100C10002C31B86903F004F83A69F8602368127B54
:100C20005869191C01960295009268312C33BA69F3
:100C300003F066F9FB6978689D462368DA69191C38
:100C40001B6A00902C31786902F060FFFE68064351
:100C5000F6B23E6106F0AAF8051C06F0AFFB2D794E
:100C6000012D0AD19C300368002B06D105F072FEDD
:100C7000012802D0281C03F03BFE2568281C291CF3
:100C800068312C3003F016F9604A23681268E86670
:100C90000C20115E986D88420EDC0E20115ED86D1E
:100CA000884209DB1020115E186E884204DC122194
:100CB000525E5B6E934221DA00233B8420220123A3
:100CC000D35505F055FE002818D105F02DFE00285B
:100CD00014D04D4B1A68FF239168FE2901DC9368FC
:100CE000DBB22120C355381C0221203005F0DCFE88
:100CF000474804F00BFC03F0FDFCE2E7414E454998
:100D0000336802241A6858680A709A68CB78487069
:100D10007F20834380256D4223432B43CB70532395
:100D20008A700B710132BB6952009A18012005F0DC
:100D30001DFF336838491B697F204B70CB787A6977
:100D4000834323432B43CB7001206D230B7105F0AC
:100D50000DFF336820211A682120CA555968C155F2
:100D60009A682220C255591DC97F2320C1551B698D
:100D700025202421CB55C35D7F218B4323431D4375
:100D80000132C319B869520082181D70391C0092D3
:100D9000002201202031131C05F0AEFE01F0C4FF3B
:100DA00001F0E0FFFFF7B4FE002827D1164C2368BE
:100DB000586904F005FA2368D86E04F061F903F06D
:100DC00065FF396900290DD12368B9691A1C2C32D5
:100DD0001B68B86806F058F8236878681A6879695B
:100DE00006F0A6F8022003F0B1FD786906F07EFB5C
:100DF0002068703007F098FA002000E0201CBD4603
:100E00000BB0F0BDF802002000000020900C002084
:100E100010270000B803002004010020F0B5940062
:100E2000231C0A3385B0DB08DB006946C91A02AF10
:100E30008D4602AA061C7A60101C0021221C08F0B4
:100E400091F9231C0833DB08DB006946C91A8D467B
:100E500002AD281C221C002108F084F90C4C301C27
:100E60002368996A5A6A683300910193291C7B6848
:100E700007F07CFA301C01F0D5FF2368301C5A6A59
:100E80009B6A291C00937B6806F0C4FCBD46F7BD35
:100E90000000002070B50C1C151C1E1C06F004FF81
:100EA000144B201C1B68596A9A6A07F003F8201C2F
:100EB00007F00EFC201C07F0F9F8321C201C291C3E
:100EC00007F0B0F9201C291C02F088FD05F06EFF28
:100ED000041C06F073FA8E300378002B09D12379B5
:100EE000002B06D005F036FD012802D0012003F0CA
:100EF000FFFC70BD0000002038B508F019F8051C93
:100F0000012008F029F8041C281C03F0CBFA201C4F
:100F100003F0D4FA38BD38B508F0BEF808F010F880
:100F2000051C002008F018F8041C281C03F0BAFA6D
:100F3000002004F0EFF8201C03F0C0FA03F0BAFC24
:100F400038BD10B5A4B08C22041C002101A808F003
:100F500009F901A8211C07F0A1F907F0C9F901A8B6
:100F6000211C01F0C5FF24B010BD000038B506F00B
:100F700025FA294C8E30236801781A79002902D18C
:100F800051B2481C04D10025DD60AA420DD116E003
:100F9000D8681A69904202DAD8680130D86001290D
:100FA0000DD0DB6893420ADB01251C4900202B1C75
:100FB0000E33021C0B7105F0D9FD23681D712368E7
:100FC0001A79002A03D1164A1268127804E0012A1D
:100FD00003D1134A126852781A60186804F072FA42
:100FE0002368051CEC33186804F090FA2D1A002DC4
:100FF0000BDD2368186804F065FA2368051CEC33E0
:10100000186804F083FA281A00E0012003F070FC4D
:1010100003F090FC38BDC04600000020BF03002054
:10102000900C002008B505F095FC002802D10220A4
:1010300003F0F8FF08BD0000F0B589B0061C05F00C
:10104000B5FE059006F0BAF9031C98331A68A14B57
:10105000002A08D1A0300268511E8A41D2B20492FF
:10106000002A06D001E0012004901A680021B8325D
:1010700005E01A68B8321168FE2901DC01311160FF
:101080001B6800211A1CB43211700499002904D085
:1010900091490968097D00295AD0181CB33001789C
:1010A000C9B2002908D003785BB2022B00D001231B
:1010B00013700023037070E11D1CB0352C78002CD8
:1010C00009D0012414701A1CB132BC33017029708C
:1010D0001170196062E10498002839D1191CBC31E3
:1010E0000C68002C09DD013C012C01D00C602FE0C4
:1010F000049B0B600323137050E11A1CE832126842
:101100001188764A914223D01A1CC8321188744A39
:10111000126852888A421BD86F4C2068427C181C87
:10112000B8300068904213DB07AA1180CA331B88CD
:101130006C49538002234B70CB70049815230B71BC
:1011400005F014FD634B22681B68927CBC331A6067
:10115000614C2768F87C002800D01EE104995D4DA1
:10116000002900D082E02C68231CE7331B78002B79
:1011700056D03B1C2C331B78002B51D0231C0791DD
:10118000DC331B680393231CC83303981A8843007D
:101190009A533B1C2D33197804984B00F618031C06
:1011A000994206D05A00B21A023A128801338018C6
:1011B000F6E7FEF7CDFF0790FA8B231CE033904251
:1011C00002DA1A68013200E000221A603A1C2E325C
:1011D00012781B68934215DD42497C235B42CB7039
:1011E00007AA1623012400200B714C7005F0BEFCE9
:1011F0002B6800201A1CDC32E0331060186005F008
:10120000F7FCCBE03B1C2D331A780399231C013AE1
:10121000DC33914202DA0A1C013200E000221A603B
:10122000C4340137FB7F22689A4217DB2E49002025
:101230001223021C0B7105F099FC2A682648131C26
:10124000C03319680068013119600230C07F8142E3
:1012500004DB00211960B432022313702A680023D2
:10126000111CB231C4320B70136047E02B681A1C9A
:10127000BC3210602A321278002A3FD0191CC831C3
:10128000098807AA1180CA331B8816495380022394
:101290004B70CB7019230B7105F068FC2B6822682A
:1012A000191CC8310C88D08B163984421ED2181CE8
:1012B000CA300488508D844218D2097800291DD183
:1012C000C43301321968D27F914217DA01311960B3
:1012D00014E0C046000000208C0C0020FFFF00003E
:1012E000900C002004010020BF03002001220A709E
:1012F000191C0022C431C0330A601A60294D2B68C2
:101300001A1CE6321278002A47D105980279002A81
:1013100041D01A1CB0321478002C3ED1224ED86A2B
:101320003768798BBA8BFB8A3F8B009705F0F6FC08
:1013300036682B68718CB28C071CD86AF38C368D9A
:10134000009605F0EBFC2B681A1CC8321188CA33D2
:10135000B94202DA1A88824210DB07AA11801B8880
:101360001249538002234B70CB70002017230B715E
:1013700005F0FCFB2B680122B1331A702B681A1C94
:10138000B1321278002A08D00499002905D0B03370
:1013900001221A7002E0B1331A700124201C09B036
:1013A000F0BDC046000000208C0C0020040100208D
:1013B000F0B591B002AF03F06FF8061C03F084F8AB
:1013C000386103F075F8B04BB8601C686846E36894
:1013D00000211A1C0E32D208D200801A22698546DA
:1013E0000E32D208D200801A02AD8546FD6102ADF0
:1013F0007D6272799A18131C0E33DB08DB00C01A69
:1014000053000E33DB08DB008546C01A02AD85466B
:10141000C01ABD6102AD854602A87861B86907F0BF
:10142000A1FEE1687279281C52180121520049423C
:1014300007F098FEE36872799449D21852007869EF
:1014400007F090FEE2683969F8693D6307F048FEED
:1014500039692269BA31FF31786A4024002507F0E2
:101460003FFEFC603D62796AF86904F0EDFE0320FE
:1014700003F000FE844D86492B68864C5A68186834
:101480004A709A680423CB7051230B7123688A70C9
:101490005B690132920008709A18022005F066FB21
:1014A0002B687D491B6904254B705A230B712368F7
:1014B0000220DA69CD7005F059FBB479013C631C58
:1014C0002CD07579013D6A1CF8D073797869634333
:1014D000EB185B001A5A714B9A42F3D0B96930226B
:1014E0007960F9627863D219694609CA09C1211C79
:1014F0007B68F8692A1CFFF72FF8002803D03B6AA5
:1015000001339BB23B627379BA6963433869EB1864
:10151000D15CC25C8A18F969CA54D3E7F479013CFA
:10152000601C2FD0B17973797D694B43E3185B0060
:101530005A5B5A4B9A42F2D0BD6930207D60FD6201
:10154000C0197D6984467D636846624628CA28C002
:10155000221C7B68786AFEF7FFFF002803D03B6AF5
:1015600001339BB23B627379B279BD695A432B193F
:101570003D699A5C2919BA31FF310B787D6AD3181D
:101580002B55CCE7404B3C6A1B68DA681B69D318C3
:101590009C4206DAFB68013BDBB2FB60002B00D00B
:1015A00061E73B4CB3797F252370737980206370AA
:1015B000A370E3784042AB4301252B430343E37020
:1015C0000820D223211CFA69237105F0CFFA324991
:1015D000F3797F224B70CB78082093431D438023FF
:1015E0005B421D437A6AD323CD700B7105F0BEFABE
:1015F000B379251C013B0FD37279013AFAD3717983
:10160000FC69594389186118BC68E01864300C788B
:10161000007820180870F0E7F379013B08D3BC6824
:10162000E2187C6A7C321178E25C8A18E254F4E7B2
:10163000F869796A04F008FEB3797F202B7073791A
:1016400001216B70AB70EB78802483430B436442C1
:101650002343EB70291C1D23FA6908202B7105F028
:1016600085FA0D49F3797F224B70CB78012593439E
:101670001D432C431E2308207A6ACC700B7105F0A1
:1016800075FABD460FB0F0BDF8020020FFFF000064
:10169000B80300200000002004010020FEFF00002D
:1016A00008B502F005FF58300378002B02D1FFF790
:1016B0007FFE01E003F0D4FE08BD0000F0B591B05C
:1016C00002AF05F029F9041C07F07CFC07F0AAFC26
:1016D00001F026FBFFF788F805F01EF9061E062E1E
:1016E00000D1C6E0062813D8022800D17EE005D834
:1016F000002823D001286CD0341CEDE7042800D149
:10170000A5E000D9ACE005F063F9FFF7C9FF99E067
:10171000092800D1CBE007D8072800D1B3E008287A
:10172000EAD105F055F9B8E00B2800D195E100D2D7
:10173000CFE00C28E0D105F04BF997E105F00AF96C
:10174000002812D00128D7D1CB4D02222B6819696D
:10175000186AB961C949F8611A621E61301C3F23D9
:10176000321C0B7105F002FA22E00125012D02D096
:10177000022D0AD00FE0002000F084F903F0A6FA51
:10178000C0B205F041FAFFF78BFF0020211C021CBC
:1017900000F034FE051C05F0DDF80028ACD105F0A2
:1017A000BBF80028E2D0A7E705F0B6F800280AD178
:1017B000FFF776FF211C0122002000F0F1FE05F06A
:1017C000C9F80128F0D02B68FC691C62BC691C6157
:1017D00092E705F0FDF805F09FF80128FBD007F02F
:1017E000CFFBFFF701F804F087FF85E7FFF784FBE5
:1017F00005F058F8002003F08DFC03F055FCFEF7CF
:101800007DFEFFF74DFF05F0E3F805F0EBF8042847
:101810000CD004D800280ED001F0A6F80BE0052863
:1018200007D0062807D103F045F804E004F0A2FD34
:1018300001E003F02DF805F06FF80228E5D0FFF77E
:101840006AFB59E705F068F80328FBD054E705F078
:10185000BFF801F087F805F05FF80428FBD04BE7EC
:1018600005F0B6F803F040FD05F056F80528FBD06A
:1018700042E705F0ADF8022000F004F905F04CF85D
:101880000628FBD038E705F0A3F8012000F0FAF8AD
:1018900005F042F80728FBD02EE7002003F0EAFB12
:1018A00003F046FC05F038F80828F6D024E705F0E8
:1018B0008FF8002002F0F4FE002003F0DBFB03F0C1
:1018C00037FC05F029F80928F6D0012002F0E8FEDF
:1018D00012E76C4600203C6107F0D8FB07F0A2FB42
:1018E000002003F017FC644C694623685D681868A3
:1018F0001B694543EB180733DB08DB00C91A8D462B
:1019000002AAFA6102F0C8FD02F0DEFD02F0D0FD8D
:10191000FB695D19181C291C7D6103F06FFD2368AC
:101920006C465A681B69D3189B000A33DB08DB003E
:10193000E41AA54602ACBC6105F04AF84E4C2020E2
:10194000236819681A79C15521202221C255CA5528
:101950005A1DD27F1B6923202421C255CB55252235
:101960000123D355FB690022391C00930420131C6A
:10197000203105F0C1F87969F86904F065FC0020B0
:1019800003F078FB23683E485C6805687C600021B2
:1019900039603A687C68A24208DA3A68A96992001C
:1019A0008958BC69A15039680131F1E7A200BC69CE
:1019B0001969A41805683960A44600223868824273
:1019C00006DA296A90000958644621500132F5E789
:1019D0001A682821CA5578689A6829242A21E0556E
:1019E000CA550533DB7F2B24E35504242D233968A6
:1019F000DC55234B01321B6892005B692C209A183E
:101A0000C1550092391C0022131C0220283105F018
:101A100073F801233020C355174B31211B68322046
:101A20001A79CA55C2555A1DD27F1B693321CA552E
:101A30003422D3553523DC55BC690022391C1020D3
:101A40003031131C009405F057F804F065FF0A28A4
:101A500000D173E73C69A5464EE604F0B9FFFEF7F6
:101A600003FE04F059FF0B28F9D045E604F054FFBB
:101A70000C28FBD040E6C046F8020020BF0300203F
:101A800000000020F0B5DA4C9DB0236800AF9B68E1
:101A900038637B625B000133BB6503F00BF923689D
:101AA000FF229B687866D31A984200DD7B66786EC9
:101AB0007C6A041B3C626C4603F002F97C65BC6DD9
:101AC000684665002B1C0833DB08CA4CDB00C01AD3
:101AD000012363707C235B423A1C8546E370211C22
:101AE000B1230020643223716E4605F03FF80023D5
:101AF000211CBC6DA34205DA3C6A5A001819B05289
:101B00000133F6E70223CB70321CE4B263230020DA
:101B10004C700B713C6405F029F82B1C7C6D08336C
:101B2000A546DB08DB006846C01A8546C01A6C462D
:101B300085467C65F86303F029FCB861012002F05A
:101B400067FF00212A1CF86B07F00CFB786D002161
:101B50002A1C07F007FBBC6D6846A400231C0A334F
:101B6000DB08DB00C01A8546C01AFC6178636C464E
:101B70008546C01A8546BC636C467C61BC69A4007E
:101B8000BC600024BC640021FA69B86B07F0EAFA73
:101B9000786BFF21FA6907F0E5FA0024944BFC65A5
:101BA0001B68FC6D5B689C4251DA3C6A0026E4B21B
:101BB000201C7C6403F08FF803F05CF802F01EFF39
:101BC0007C697D6B3C61BC6BB86D0136F217C30F4D
:101BD00086425341DBB2FB62002B06D1796C881937
:101BE000C0B203F078F803F045F86B46FB60BB68C1
:101BF0006A460A33DB08DB00D01A85466A46FA6477
:101C000003F0CAFB0020031CBA69934205DAF96CA1
:101C10009A008A5801338018F6E72368984200D961
:101C200020602968884200D2286002F0DBFE3A6911
:101C3000043501C23A61FB68F86A9D460434002805
:101C400002D102F0DBFEBFE7FC6D0134A6E7002401
:101C5000694DFC65BB6D9C4217DAB96B7A6BA300CA
:101C6000C858D358C01A854204DD3B6A051CE318E6
:101C7000BB623C65F96D814200DAF86502F0B2FEA4
:101C80007A6D6300D0520134E4E7F86D02F0AAFEE9
:101C9000574B1B685B88984206DA3C6B012C03D0DB
:101CA0007C6EBC627C6A3C65544D00262C683222F6
:101CB000231DDE670433DA67803364221A60396DCE
:101CC00001220220DA607A6B81408A5898605E6057
:101CD000101C7A60796402F085FE98347B6CB96BD5
:101CE000206058582C6802F07DFE2B68A0342060DC
:101CF0001A1C01213C6BAA324942AE3311801E806E
:101D0000012C22D1FA6B331CBC6DA34209DA7C6D25
:101D10005900615A1088884200D211800133023282
:101D2000F2E73C6D6300FC6B1A5BBC6C131CA242B7
:101D300000D2231C2F499BB23C6CBB6400200223C1
:101D40004C70CB700871FA6B19E0386B294C022883
:101D500008D1396C04236170E3702671301C211C9A
:101D60007A6926E0F86D02F03DFE3A6C80B262704E
:101D700002237A6DB864E3702671301C211C04F0D4
:101D8000F5FE386D6824E053BC6A6A21CC537C6D43
:101D900043001B5BBC6C6E216C20CC531549C353B4
:101DA00004234B700223CB703A1CB2230B7100202A
:101DB000683204F0DBFE3C6D63007C6D1B5B0F4CF6
:101DC0002268111CE83109680988994223D207F07A
:101DD00063F9051C07F0C8F80378061C002B0FD028
:101DE000012004F005FF23680236E8331E6023E07B
:101DF000900C002004010020FFFFFF7F0000002066
:101E0000002D19D1174B1B68DB7C002B14D101204E
:101E100004F0E2FE10E0E7321278002A0CD0124DF6
:101E2000286842889A4207D9002004F0E1FE23681E
:101E30002A68E83302321A603C6B002C06D1BC6A77
:101E4000E0B202F048FFBD461DB0F0BD04F064FDF5
:101E5000072800D197E604F05FFD062800D192E63E
:101E6000EDE7C0468C0C0020900C0020F0B585B04A
:101E700000920391029007F00FF9061C04F088FD10
:101E8000071C04F08DFD734D01902B681A1CE43281
:101E90001278BA4220D0002F08D06F4900203B238F
:101EA000021C0B71022604F061FE10E001993C1C3B
:101EB00000290DD168493C23381C3A1C0B7104F0F1
:101EC00055FE2B68E6331E78731E9E41F6B2012440
:101ED0002B68E4331F701DE01A1CE532127801995B
:101EE0008A4216D0002906D1E6331E78731E9E4121
:101EF000F6B23A2301E03923022657490020021C9A
:101F00000B7104F033FE2B68019AE5331A7001243B
:101F100000E0002404F010FD071C04F031FD009BDC
:101F2000032B02D0002F03D107E00124002F36D06D
:101F3000002004F009FD012431E02B68E4331F8800
:101F4000002F2CD10099012902D0022904D00EE0E3
:101F5000009804F041FE0AE0381C04F03DFE2B68B6
:101F6000E7331B78002B02D0381C04F041FE04F04C
:101F70002DFE2B68071CE6331B7883420FD0002808
:101F800002D01123012601E01223061C3249002051
:101F9000021C0B7104F0EAFD2B68E6331F7007F09A
:101FA0007BF8B04239D007F077F806F0C9FF071C7C
:101FB000301C06F0C5FF009007F06EF8301C07F0EB
:101FC00065F807F02FF8254B1B681B7D002B10D000
:101FD000012C0ED0009B3A1C5B325B3303990298B4
:101FE00005F010F8002003F045F80024FEF714FC7B
:101FF00006E02B680020CC33187003F08BF8012426
:10200000002004F0F5FD2B6800211A1CE732117046
:10201000134AE833126802321A6007F03DF806F0FE
:10202000A3FF0378002B08D004F0DCFD2B68E73316
:102030001A78824201D01870012404F0B9FC051C02
:1020400005F0BCF90379AB4200D00571201C05B046
:10205000F0BDC04600000020BF0300208C0C002013
:10206000900C0020F7B5434C151C236801911A1CF5
:10207000B1321278061C002A23D01A1CE6321278DC
:10208000002A1ED11A1CCC321178002919D1B03384
:102090001B78002B15D10123137002F009FA071CDD
:1020A00002F0FAF93A1C031C5B324533301C0199EB
:1020B00004F0A8FF02F0AAFF022002F0B3FFFEF72F
:1020C000ABFB23681A1CCC321278002A4FD01A1CA2
:1020D000294F0020B03210703A680190126A011C3A
:1020E000013A0ED30E265643B446AC446646B68833
:1020F000002EF5D036B20131B042F1DA301C019237
:10210000EEE71A1CE6321278002A13D1012911DDFC
:1021100005F054F90123983003603B681B6A013BCA
:102120000AD3019EB342FAD00E225A430021AA18C4
:102130009180F4E7002904D023680022D4331A6088
:1021400008E01A1CD432D03311681B68994201DCB4
:10215000013111602368191C1A1CD431D03209686E
:102160001268914205DDB03301221A7001E0D433C8
:102170001A60F7BD00000020F8020020F0B5984C6E
:102180008FB002AFFA612268FB60136892689D1CF1
:10219000520055437960694639605208291C013361
:1021A00053430831C9088F4EB860C9006846401AC9
:1021B00085460133306802A95B00CB18B9613C2227
:1021C00000212C307B6106F0CDFF2A1C0021B8696C
:1021D00006F0C8FF84490020A623021C0B7104F0FE
:1021E000C5FCFEF7C3FE3168081CC830CA31FEF7D3
:1021F00037FB23687D4D5B6804226B705B232B717A
:102200003368EA7002209A69291C04F0AFFC236845
:1022100002201B69291C6B700423EB706C232B714B
:1022200033681A6A04F0A2FC23682020196821226E
:10223000C15558682221D0559A682320CA55591D86
:10224000C97F1B69C1552421CB5504202523D855AE
:10225000336801325B6992009A180092391C00229F
:10226000131C0220203104F047FCB8687968BA6971
:102270007B69FEF797FCB861002800D08DE02668E6
:102280006A46F36A3A611A01131C08336946C81A90
:10229000854602ADB969281C06F064FFF26A281C65
:1022A000F969FEF7BBFD236869469A6A0E235A4313
:1022B000131C0833DB08DB00C91A8D4602ACB96970
:1022C000201C06F04FFFFB68281C211CFA69FEF752
:1022D000E1FDB86CFEF7B0FE454B1B681B7D002B83
:1022E00004D1B8687968221CFFF7BCFE201CF9698C
:1022F00000F08CFF201CF96900F0FAFD06F036FBB7
:1023000083000733DB08DB006A46D21A954602AB2E
:10231000FB60334B061C1D680E22A86A7E61031CFD
:10232000013B5343E418F8610434F8690138F8615B
:102330000FD30021635E002B09DD7A69FB68013A47
:1023400090007A611818211D042206F0C9FE0E3C87
:10235000EBE768682A682923D8552821AB68CA5555
:102360002A21CB550535EA7F2B20C2552C2100228E
:10237000CA551C49013309687E22896A5B00CB1863
:1023800052422D20C255391C00932831F2B203204D
:10239000FB6804F0B1FB39698D463A68954602F056
:1023A00013FD02F033FE02F0FBFA012002F062FEA0
:1023B00002F036FC0B4BB4221B68B8689A56796859
:1023C000FFF754FD002800D1B8690A4B1A680A4B80
:1023D0009A4202D002F088FFFEE7BD460DB0F0BD84
:1023E000F802002000000020BF03002004010020AC
:1023F0008C0C0020C40C0020CDCDCDCDF0B5494CC7
:102400008BB0236802AF1D68B96059687A604D438C
:102410000A229A621022DA621B696A46EB189B0054
:102420000A33DB08DB00D21A954602ABF860BB61C9
:1024300004F0CAFF236869469C6AAD00E200131CE1
:102440000833C91A8D4602ABA400FB61231C083374
:10245000DB08DB00C91A8D4602A93961F869002141
:1024600006F080FE221C0021386906F07BFE2E4E0D
:10247000002433686946F0331C702C4B1B682D33E5
:102480001A785200131C0833DB08DB00C91A8D468A
:1024900002AB181C211C7B6106F064FE04F07AFC80
:1024A000B969BA694D192B1C4178201CFEF792FAC4
:1024B000BA68FB689A4201D004F08AFA33689C60DB
:1024C00004F09CFB041C02F001FCA04204D0201C80
:1024D00002F001FC02241DE079690091FA69291CCF
:1024E0003B69B869FFF74AFE0F4B114A1B68041C91
:1024F0009968914202D09A6801329A60002809D105
:1025000004F028FA7A68904204D104F005FAFB68D6
:102510009842D5D0F869FEF714FD201CBD4609B0DD
:10252000F0BDC046F8020020000000208C0C002006
:10253000FFFFFF7F184BF0B51B6885B01E689B68D6
:10254000B41C5B005C4300AF221C5B08FB600832DC
:10255000124BD208B86079601868D2006946891AAF
:102560008D463C2200212C3006F0FCFD221C6846E2
:10257000002106F0F7FDFA68731C534301336D46E2
:102580005B006A46EB18B8687968FEF70BFBBD463E
:10259000C0B205B0F0BDC046F80200200000002027
:1025A000F0B5B74EE9B0336802AF1D68F9615968FC
:1025B00005244D437A6002229A62DC621B69B8608E
:1025C000EB1893400A33DB08DB006A46D21A9546C3
:1025D00002ABBB6101F07EFF04F0F6FE381C002167
:1025E0001022483006F0BEFD0023BB63FB63336856
:1025F00069469A695B69AD0053439B000A33DB0867
:10260000DB00C91A8D463B1C02AA58337A613B6431
:1026100004F0C0FB061C03F039F9BB69201C5D19EE
:102620003D611A1C71782B1CFEF7D4F903F08EFC67
:10263000944C786923685969FEF718FAF969BA6801
:10264000914201D004F0C4F98F490020A223021C5A
:102650000B7104F08BFA236800249C60FC617C629F
:1026600004F0CCFA386202F031FB3B6A984204D0A5
:10267000181C02F030FB022664E1002C72D1804B62
:102680006A461B68FA609A6951005A6901324A43E6
:10269000131C0833DB08DB006946C91A8D4602AEFD
:1026A000301C211C06F05EFD7A6A764D082A08D19E
:1026B00003F04CFC2B6878695969FEF7D7F97C6206
:1026C0004CE0042002F0D6FC2B68301C59697A6972
:1026D00004F030FD051E012D0FD103F0D7F80520C1
:1026E00002F0C8FC6849A323201C221C0B7104F0D3
:1026F0003DFA00232C1C7B6230E0644D311C2B68BA
:10270000786933331A7804F0D9FD2B68F9693333CB
:102710001B785B0099420ADD03F0B8F8052001211F
:10272000BA693B69FEF756F903F010FCFC61FA69DF
:102730002B680132FA613233187802F0CCFA02F0D9
:10274000E1FA2B683333187802F0DEF8002002F04B
:10275000FDF8386A02F0BFFA02F0F8FAFB680026CA
:102760009D46D9E0494B01241B6834331878454B0A
:102770001B68186002F0C8F8052002F053FCB86925
:102780003969FFF7D7FE061E00D0C5E03C4D6A460A
:102790002C68FA60E36A69461A01131C0833C91AE7
:1027A0008D4602AB181C311C3B6206F0DBFC391C69
:1027B000E26A386A4831FEF731FB2B6869469A6A4B
:1027C0000E235A43131C0833DB08DB00C91A8D465D
:1027D00002AD311C281C06F0C5FC3A1C3B1C4832DB
:1027E0003833386A291CFEF755FBA91C281C06F053
:1027F00015F8281C291C0E30103106F00FF8391C72
:10280000281C40317A6A06F0D9F87862032803D090
:1028100007282BD1182405E0381C403006F026FB91
:10282000041E26D004F09EF8184B1B689B6B1840C2
:102830000123A340034219D02C2302212D22D819B1
:10284000D955D45504F030F902F0E0FB012002F034
:102850004FF80D490020A223021C0B7104F086F9E9
:1028600003F074FB082300247B6253E0796A082993
:102870000ED002F0CBFB012402F0A6FA4AE0C046DB
:10288000F802002000000020BF0300208C0C002074
:1028900004F096F800282ED00224381C221C2D4962
:1028A0002C3006F01DFC381C211C2C3004F0FCF8E8
:1028B000052004F01BF94422D35D3021CB5532238F
:1028C000DC55312200233321D455CB553422352118
:1028D000D355CA5D7F218A43144380225242144358
:1028E0003522D4553A1C5832391C0092052030311B
:1028F0001A1C04F001F902F089FB012001F0F8FF35
:1029000015490020A223021C0B7104F02FF903F0DB
:102910001DFB0024F9688D46104B114A1B6899680D
:10292000914202D09A6801329A60002E0AD104F0D6
:1029300011F87A68904205D103F0EEFFBB68984227
:1029400000D18DE602F062FB02F0A0FF301CBD4614
:1029500067B0F0BDA0910000BF0300200000002080
:10296000FFFFFF7F70470000F0B5D74D9BB02B688D
:1029700000AF5C68061C3C64640018687C653C6CB5
:102980006043021951000831C908C900F86368465C
:10299000401A8546F8623C6C90000A30A400C008DA
:1029A0007C63C0006C460732241AD208601AD20039
:1029B000A5468546801A3C65DA686C460021854646
:1029C000BC63386206F0CEFB2B68F86B1A690021F5
:1029D000684406F0C7FB2B680021DA68386D920066
:1029E00006F0C0FB2B68F86B1A69396D8400920001
:1029F0000819002106F0B6FB2B68B449DA68B86BF9
:102A0000520006F0AFFBFA6BB96B50004308FB6154
:102A10002B6808181A69AD49520006F0A3FBFDF7B0
:102A200055FD022E05D0032E05D02F30012E05D1E5
:102A300002E0303000E03130007878647D6BAD0822
:102A4000BD617D6D6D08BD627D6C013D7D633D6D39
:102A50002C197C62FC69FD6A6300EB187B617D6B5D
:102A6000994C013500D1C1E0002002F003FB984BE6
:102A700025681B686C683B63013C64D3A0002B682D
:102A8000B864591E7965F7D3A9683A6B4B43E318CC
:102A9000013352699B009858022E0CD0032E24D08B
:102AA000012E4ED13B6BB96C9B69FB605B58C01A21
:102AB000C343DB1718407A6DBB69396D5343E31884
:102AC0009B0059583A6D401898507B6B002B38D1B9
:102AD000796DBB6A4B43E3185B00796CFB64FDF7CF
:102AE000E9FAFA6CFB6AD0522BE0796DBA694A4375
:102AF000A31899003B6DC958031E8B4200D20B1CD2
:102B0000396DA21892005350796DBA6A4A43A118E0
:102B10009446BA6B4900895A884200DD081C614618
:102B20006218B96B5200505280B21B1A7F22FD2BE3
:102B300001D85B08DAB23B6A786D19193B6C4343E4
:102B4000CA547B6D9DE72D69614B7D651D687B6D6A
:102B5000FA69013B9C00B86B9B185B00C3183B6390
:102B60007A6D013A7A653DD3E9690859022E09D098
:102B7000032E17D0012E30D12A6A1359C01AC3432D
:102B8000DB1718407B6A796A1B597A6BC0180851A9
:102B9000002A22D1796CFDF78DFA796D7A694B00A4
:102BA000D0521AE07B6A1A59031E934200D2131CBA
:102BB000796A0B51396B0A88904200DD101C3A6B20
:102BC000108080B21B1A7F22FD2B01D85B08DAB27D
:102BD000386AF96B4318786D1A54396B043C023922
:102BE0003963BDE77C6B013C7C6338E7FD6A7D643B
:102BF000022E06D0032E61D0012E6DD100F0DCF83C
:102C00006AE001F049FC381C32491022583006F0C5
:102C100067FA02F051FC21682D4B0E683864BD6ADA
:102C20001868331C013B5D433E6584467D653E6DFF
:102C3000013E3E6522D34B687E6DFD6AF018400070
:102C40005E002818FE630022023A013B11D33D6C5E
:102C5000FE6B6D00FD646546AD69B618BE64760016
:102C60007659FD6C5835ED5BAE1B855A751985524A
:102C7000EAE77E6DBD6A761B7E65D8E70B69FE6963
:102C8000134AF118FE6A49005800156871187865F2
:102C90000022023A013B0ED37E6DB0182E6A40002E
:102CA00080598E5A361AB4463E6C70005830C05B5C
:102CB00060448852EDE700F080F80DE03D6A7D64E5
:102CC00000F07CF8012308E0F8020020FFFF00007C
:102CD00000000020A29100000223226858261068FC
:102CE0005924F05511795A25E155E955511DC97FEF
:102CF0005B26F15512695C205D21C255CA5D7F21BA
:102D00008A43134380225242381C134358305D22B9
:102D1000796CD35503F06EFEBD461BB0F0BDC046C6
:102D200008B503F055FD08BD0C4B10B51B68DA6AF9
:102D3000002A03DD596B5218D10F0BE000218A42A3
:102D400008D1074909681424085F5C6B012184429B
:102D500000DB111C7433197010BDC0460000002048
:102D6000900C002010B504F013FB124B1B68D96ABD
:102D70001A1CF032002915DD041CE8342488A14215
:102D800010DA6424E630614300885C6B6043C14222
:102D900008D5191CE6310978002901D1012100E08C
:102DA000002111701278002A02D0743300221A70A8
:102DB00010BDC046000000207047704770470000FB
:102DC00008B502F071F901F0A5FC01F03FFC01F03B
:102DD000F3FB0F4B1B681A7A0E4B1B689433002AC7
:102DE00001D0022200E003220B491A6000230B707D
:102DF0000A49A0220B700A49D2050B709363D36B6A
:102E00003F218B43D36362B602F0CCFF08BDC046BE
:102E10009C0C0020FC0000202900005028000050DD
:102E20002A00005038B5041CFDF762FB051C04F0B5
:102E3000AFFA291CF0310B78002B24D0124B002262
:102E40001B68DB6A013B07D3180120180825405F87
:102E50000028F7D10122F5E70C4B1B68D86A00283F
:102E600011D15D6B002D0ED1F433002A0AD01A68FF
:102E7000FE2A01DC01321A601B68052B03DD0023EA
:102E80000B7000E01A6038BDF8020020000000203E
:102E900070B5051C0C1C161C03F0CEFD002802D0DA
:102EA00001280AD023E00E204643AD19EA88FF230B
:102EB000FE2A00D8D3B2637119E00E20704328189F
:102EC000C288FF23FE2A00D8D3B263710B220A23E3
:102ED0008256C3560921D31A0822415682568A1AAD
:102EE000934202DDA371E27101E0A271E37170BD52
:102EF000F0B5C14B8DB01B6804909E689F69069623
:102F0000DE68079103961E6905965E69029603F0D6
:102F100099FDBA4B01261B68E4331B780196002B00
:102F200058D00026079D049C0196B54B1B681B6A70
:102F30009E424FDA2B8809A803806B88438005F0F6
:102F40009BFC0420235E002B40DD238869460B8414
:102F5000638808A84B8405F08FFC68462023C35E75
:102F6000069999420BDA039A9A4208DD68462222B2
:102F7000825E0599914202DA0298904221DC042196
:102F80006A5E002A1ADD9F4A126892192832127866
:102F900052B2012A12DD0698C21B9A420EDA039938
:102FA000CA199A420ADD6A462223D35E0598C21BDB
:102FB0009A4203DA0299CA199A4205DC0023A380D7
:102FC00004E00122019201E001230193013608355A
:102FD0000E34AAE70126049C079D0296884B029FA7
:102FE0001B68013F186A874200DBB6E02B8809AEF8
:102FF00033806B88301C738005F03EFC0420235E18
:10300000002B00DC80E0238869460B84638808A8D5
:103010004B8405F031FC6B46598C1A8C794B03912B
:103020001B683088DB1960331979774B84467688C2
:103030001B68002901D14C3300E04D330420295E88
:103040001B78002911DD039836B201B2891BCE1717
:1030500089197140994208DA664630B211B2091AEC
:10306000C8170918414099426DDB019E002E6AD0B5
:103070000AAE3378802149421943DF200140207B8A
:103080000123184040231943102399438C46029989
:103090000F231940059100016146084305999843A3
:1030A000014310B2001218403170717805900398F6
:1030B00099438C4601B2091209010598B270039A2E
:1030C000069161460843F2700699A28803401943AD
:1030D000131C12B27170FF2A00DDFF233A1C049802
:1030E000311C3371FFF7D4FE301C03F0B5FC042310
:1030F000EA5E444B1B68DF196037002A01DD0123BB
:1031000000E000233B711AE004202B5E002B1ADD47
:103110000AA80023029A43600F231A4040210A4361
:1031200002700127F75772883188F6783B4076B2F3
:1031300036011E4346708170C27003F08DFC2388F7
:103140002B8063886B80A388029EAB80E388013666
:10315000EB8002960E34083540E71B690F255C1E94
:103160001D40284E621C2FD031686700CB191A1CF5
:1031700078320020125E6E33002A0FDC1B881AB2F0
:10318000002A16DD00210AA80A9141608021294306
:103190000170FF2A00DDFF23037108E000215B5E60
:1031A000002B06DC0AA800230A934360057003F095
:1031B00053FC3368013CDF193B1C6E373A88783387
:1031C0001A80013D0F23CBE7336801201A1C983287
:1031D00011680832002902D11068441EA0411C1C4D
:1031E0008E3420701268181C9C30A43301601A6061
:1031F00003F046FC0DB0F0BDB80C0020000000202C
:10320000F802002000030020B40C002070B5124B1F
:10321000051C1B680C1CEA331B78002B1BD00F4AC3
:103220001368161C191C9C310968002905DDA4339C
:103230001B68002B01D105F05BF833681A1CA4321F
:103240001268002A07DD9C331B68002B03D1281C61
:10325000211C05F023F870BDB80C002000030020ED
:10326000F0B591B00E91089003F0A0FDBC4B012188
:103270001B680E201A1C5A321278089C91401A1CA6
:103280005B3212785C33891A1A7800258B1ADBB20C
:103290000F93B44B09951B680A950C93A8330D93B3
:1032A000B14B1B681A6A5043111C23180E3B01399D
:1032B0000BD3DC88099EA64200DA09940427DC5F60
:1032C0000A9DA542F2DA0A94F0E7089E013A301806
:1032D000083807920590079F013700D1B7E0059F96
:1032E000023F00203B5E0697002B00D1A8E09C4ED9
:1032F000059C336820881A1C4E32196915782433CE
:103300003A3A03F01CFD041CFDF7F2F8F0300378A4
:10331000002B05D0336835331B789C4200DA1C1C27
:1033200033681A1C4F321278002A01D1642245E01A
:103330002A1C0C9D5D35FF35287800281CD1069F7E
:1033400064210026BE5F171C714367438C460C99AD
:103350005531FF31BC450DDDA6420BDC834F0E68B5
:103360003F6801360E60DA373F78BE4204D101264D
:103370002E7000E0002008600C985D30FF3001786E
:10338000002915D0069E0C990025755F5531FF3137
:10339000A5420BDD0D681E1C01350D603E363678EA
:1033A000B54205D1002505700D6001E000200860E0
:1033B0000C995D31FF3109780029B7D06949079F21
:1033C0000968069DC819283006780020285E002E5E
:1033D00005D01D1C3E352D7876B2AE421ADC642530
:1033E00045435443A5420FDB1A1C44321278099F0F
:1033F000059E7A4334889211944205DB9B6C0A9CAB
:1034000063439B1198421BDA059D069E00232B8087
:1034100033800CE034331B78554D5C436843624382
:1034200090420DDA059F069C00233B802380079A7B
:103430000E3292008A18983153600B68013B0B6082
:10344000079D059E013D0E3E0795059643E7454BBA
:1034500000221B680E9D98331A60434B1B681B6A41
:103460005C1E0594059EE2000E247443AF18089D6F
:103470000C2272432C193F330C9D0D9E5B00EB1800
:10348000B218AA3307920993059E364D013600D132
:10349000FEE10426A35F324A002B00D1B9E1059E6C
:1034A0002D681268A9190B1C283318783E32013098
:1034B000C0B21870127840B2961DB04201DD0432DD
:1034C0001A702823CB56012B03D123883B806388B5
:1034D0007B80059EAB1928269E57012E00DC80E1DB
:1034E000B01C0321FCF78AFE0A91022E42D11E4B2A
:1034F00000203A5E1E6802217B5E69692D69306892
:103500006D10551B76688C46E917013E6D18360222
:103510004D40761B7F2E0ADD65466910591ACE177D
:103520000138891900027140401A7F280DDC002102
:10353000605E801A0222A15EC91A04F083FB0B2888
:1035400003D93B8823807B8863800323013B19D305
:103550002188079D5A00A9526188AA18D180F5E7F1
:10356000B40C002000030020F8020020B80C00205A
:10357000102700000A9E079D3A887300EB181A80F6
:103580007A88DA80D34B059E1B680221655E9B1901
:1035900028331B780020265E5BB20893032B00DCE7
:1035A00015E10A9A07985300C3181988101C0D9149
:1035B000043003210693FCF721FE079A4B00D31831
:1035C0001888DB88069A0E93089B8446D188042BC2
:1035D00008D10022B85E301AC317C018584002261E
:1035E000BB5F09E0099B0020185E301AC6178019DE
:1035F0007040099E1423F35EED1AEA17AD1855408A
:1036000023884019099D059E2B806388B24AAB82AE
:103610000C9DAB192133FF331D78002D06D01568A2
:1036200062352D88A84208DC002505E01568643560
:103630002D88A84201DB01251D701B78002B2BD1A2
:1036400012688021131C603212885E331B8800923E
:103650004A0003F063FB069D061C0020215E00204B
:10366000285E0B1ADD175A19069B6A4094460222FF
:10367000A55E06229A5EAD1AEA17AD18554065445C
:10368000321C2B1C05F07AF9069B20800222A15ED9
:103690000620185E321C78E00D9E6046B5B22B1AEB
:1036A0001BB2DA0FD3180E9A89B25B100D938B1AE6
:1036B0001BB2DE0FF3180020265E5B100896022076
:1036C000265E0E930B960D9EAB19089D1BB2EB1A4E
:1036D000DE170E9D9B19734049190B9E09B2711A92
:1036E000C817091841405B180025802B01DD1D1CFF
:1036F000803D0A9803210530FCF780FD079E764B3C
:1037000049001B687118039106991A1C0020085E75
:103710005B320F99167801321278414303980A926E
:103720000022825E0898724389180A9A42438818D8
:103730001A1C5A3212780699104104900620095E2C
:103740000F985D334843844603981B780621415EF9
:103750000B984E430A996644414376180E991641D8
:103760005943114176180D994B4313411A1C049B80
:10377000089998188022D2002B1C05F0FFF88022AF
:103780002080D2000220215E301C2B1C05F0F6F8B0
:10379000514D60802B680421785E0422A15E0433C1
:1037A0003E269A5F431ADE179B19734005F0E6F830
:1037B0002B68A080F888E18804333E255A5F431ABD
:1037C000DE179B19734005F0D9F8E08009E000206E
:1037D0003B5EF6187610268002217B5EED186D1098
:1037E00065803C4B3C491A68059D0968531928209F
:1037F0003E3118560978884203DC01225242A280E9
:1038000003E09832116801311160303300229A7060
:1038100032E02E680599126870180692021C283250
:1038200000269657B446069E3E363678B4451CDDD3
:103830000426B95F00291FD0303086780136F6B2F1
:103840008670069976B23F3109788E4213DC3B8848
:1038500023807B886380BB88A380FB88E3802B6800
:1038600098331A6801321A6006E00C9D059E1370A9
:10387000AA192132FF321370059D079E013D05955F
:10388000099D0C3E023D083F0E3C07960995FBE55D
:103890002B680022A0331A60104B1B681C69013C86
:1038A000611C00D197E0286862008218161C6E36F1
:1038B000378805970599084F002918D07823995E15
:1038C0008C4605990BB26146002909DC39683C3108
:1038D00008E0C04600030020B40C0020F8020020DD
:1038E00039683D3109788B4201DA00233380318811
:1038F0000319079300293FD08033059398788446B5
:103900007F2804D001239C44059863468370079B5D
:1039100080339B785BB2022B13DD78320023D05EBC
:103920003A6809B294460422944463463E229B5E60
:103930000593431ADA179B185340059A05F01EF8B1
:1039400030802B6802201A19111C80310856396802
:1039500040310978884207DC211C343149005B186A
:1039600001214942D98003E0A0331968013119606F
:1039700080320023D37192E73F68079B069780331C
:103980000227DF5705974027BC46069FBC44674681
:103990003F78BC46059F674518DD78321288002ABB
:1039A00000D17CE7DF79BC460127BC446746FFB203
:1039B000DF717FB2BC46069F41373F78BC4508DCCB
:1039C0003280A03003680133036068E72868031978
:1039D0008033997063E711B0F0BDC04638B5051C5F
:1039E0000C1C02F0B7FF012803D0281C211CFFF794
:1039F00037FC38BDF0B58FB0059007910A920B9354
:103A00000024404B1B68DB6A9C4278DA059F230147
:103A1000FB1808201B5E002B6FD0079FA300FB182C
:103A20000327DF5708979B78013F5BB20693049703
:103A3000089F049801370997B8425EDC069E013E54
:103A4000069B01339E4255DC2E4B04991B680131C5
:103A50009A680A9F5143481C80193D5C013D47D339
:103A6000DB6A9D4244DAAC4242D0079FA300DB5F91
:103A7000254F40003F683F89BC46149FC05B83428E
:103A800036DC069F6046C91943430131149F490043
:103A9000C95B9B118B422BDA099F7A43B218013222
:103AA000149F5200D25B934222DAA54202DB2B1C08
:103AB000251C1C1C059821010DAF41180A31381C2A
:103AC000042205F00DFB059A29015118381C0A3112
:103AD00003F02CFD00970A9F231C01970B9F05986C
:103AE0000297149F079903972A1C03F03DFD2C1C95
:103AF0000236A5E7049F023799E7013481E70FB04A
:103B0000F0BDC046F8020020B40C0020F0B585B02E
:103B10000C1C151C01930390FCF7D8FCFCF7E2FC8D
:103B200000F0BAFC384E3949336802201B692A1C60
:103B30004B700423CB705A230B7103F017F8231C2E
:103B40002A3300221A7080231B066363304BA36361
:103B500033681A692F4B19682F4B1B6802932F4B40
:103B600018688446013A43D3019F9600BF59A8596B
:103B7000C31B676B9F4200DA6363A76B9F4200DD44
:103B8000A3630B78002B06D0029FBB18BA33FF3318
:103B90001B78584380110A9FBB591B0C1B1A11D468
:103BA000487B834202DB0120664630710F200856B5
:103BB000834212DB2768181A3818206060690130C8
:103BC00060610AE011200856834206DCA668181AD4
:103BD0003018A060A0690130A061039F50003B52E3
:103BE000201C2A300678B34200DA331C0370B9E790
:103BF000084B2A341B6822781B7A00209A424041E5
:103C0000C0B205B0F0BDC046F8020020040100209B
:103C1000FFFFFF7FA80C0020AC0C0020FC0200205E
:103C2000F0B595B013930C1C0C921290FCF74EFC5F
:103C3000FCF758FC964B1B68F0331B78002B06D121
:103C4000944B1B681D7A0A950A27DE5F05E0924BAC
:103C50001B689D780A950427DE5F904D90492B687C
:103C60000C9F5A6818684A709A6804238A70013257
:103C700092000870CB70BA18512302200B7109967C
:103C800002F074FF0023A21D8248D3770232D3775B
:103C90007F262968621D05688248D677E21DD6779F
:103CA00000684A680F908048013AD2B200680E92CC
:103CB0000A6810907D4E8020013A000652B2AC4650
:103CC0000896079006930493002A00DAA3E00E9F5B
:103CD00050007BB20B90002B00DA9AE08E68551CE6
:103CE00075430135ED18A8000C9F0195139D9E00AA
:103CF000C059AE59079F861BB74200DA0796089D48
:103D0000B54200DD0896664637784E68002F09D028
:103D1000351C55430F9FFF187F5D109D7843AD689C
:103D20006843001356431A9F9E19B600F659129F16
:103D3000360C301A019E7500E8536646002854DBA5
:103D40000F257557A84212DB2768451B7D19256092
:103D50006569102701356561F757F67B656876B2AE
:103D6000B84201DC861B00E0BE1BAE196660E56848
:103D7000A84204DDDEB2D7B211960D97E060664628
:103D8000357BA8421BDB251C08351F26AE579E42FB
:103D900000DAEB77E51D1F26AE579E4200DDEB777C
:103DA000A51D1F26AE57964200DAEA77651D1F262D
:103DB000AE57964200DDEA77069F0137069785B237
:103DC0001C9F5E000295BD5B029F7D192F1C1C9DF0
:103DD000AF531B9D0B9EAF5B029EF5191B9F0B9E65
:103DE000BD53049F3F18049711E011257557A84251
:103DF00006DCA768451B7D19A560A5690135A5618D
:103E00002569A84200DA2061049E361A0496013B17
:103E100061E7013A58E7214B04981B680125D968EE
:103E2000FCF796F922497C235B42221CCB70E061AF
:103E300076231C32281C0B714D7002F097FE069FF2
:103E4000A21D27621F21631D51561F229A56164B31
:103E50001B68914201DB1D7101E000221A71079D70
:103E6000089EE562119F231C0D9D283326631F7059
:103E70005D70E6680A9F0120BE4205DA2369099D4C
:103E8000D80FEA179D425041C0B215B0F0BDC046F0
:103E900000000020A80C0020B00C0020F802002038
:103EA000B8030020AC0C0020FC020020FFFFFF7FC5
:103EB0000401002007B5104B2A301B680278987C5B
:103EC0000968424392098A4200DA0A1C997B4A43F4
:103ED000921101921B7B9A4200DA01930749012358
:103EE0004B707C235B42CB7006201F2301AA0B7111
:103EF00002F03CFE01980EBDA80C00200401002039
:103F0000F0B591B0099316AB1B78BE4C0F9300230C
:103F10004B72CB720C907F2320680B728B720691D0
:103F20000A920323C3562027FF1A0223C356099976
:103F30007F00FF1A49687F10FFB20591079704229E
:103F4000815E0623C25E0823C356407A40B20090C9
:103F5000059802F0E3FEAC4B80021D682968FCF76F
:103F6000F7F824686A682378002B00D16EE0189D6A
:103F7000911CEB8849006B802B892E1C2B800B1F1A
:103F8000EB181D887552991E0988D980617800291F
:103F900003D0079D6FB27F0039E0023B013A39D36D
:103FA0005E88DD88032161567519079E4D431F8881
:103FB00071B21E89BE194E430221AD1961569E8809
:103FC000714369188911414309141981E5E70325F3
:103FD00065575988DE886D00AC460D1CB14200D291
:103FE000351CADB266466E431D89B4461E88311C31
:103FF000AE4200D2291C0225655789B29E887943BA
:10400000754361444D19AD1145432D141D81023B8B
:10401000013ADCD2099F0B207F68049720560422C6
:10402000A15E0623E25E0A23E3560090381C02F0EC
:1040300075FE754B80021C686168FCF789F8714B4E
:1040400021681B681A78002A0CD164E0531C189F61
:104050005B00FB18013ADDD31988023B4143091488
:10406000D980F7E7179CE288251C62802289261CEC
:1040700022808C1C6400221FAA1815883553941EB8
:104080002488D4805C78002C03D0079C67B27F0022
:1040900039E0023A013939D35688D58803241C57B0
:1040A0007519079E6543178874B21689BE19664351
:1040B0000224AD191C57968874432C19A41144434B
:1040C00024141481E5E703255D575488D6886D00D4
:1040D000AC46251CB44200D2351CADB264466C43DC
:1040E00016881589A446341CAE4200D22C1C022529
:1040F0005D57A4B296887C43754364446519AD113D
:1041000045432D141581023A0139DCD21A7B002A6D
:104110000DD1079222E04A1C179D5200AA180139BE
:10412000F4D31488023A44432414D480F7E7099E58
:104130000E27D95F70680024079488420EDD102591
:104140005A5F9B7C01265BB20093231C02F0E6FDC4
:1041500010231B1A9B000B900D9307962A4B0021EE
:10416000186809910768BC4666464368711E00D20C
:104170008AE0179C4A00A2180E92013B00D281E00F
:10418000079D8468002D41D0664666430896F61860
:104190000A9F01367600BD5B5F1C2AB2D243D2175C
:1041A0002A408D1C654302967D190A9E6D00AE5F04
:1041B00012B20396964200DA0392089E341B3C1911
:1041C0000A9F6400E45F944200DA141C039E0A9F75
:1041D0003519029C3E190224375F141EBC4200DAD6
:1041E0003C1C023E2D190027F45F161EA64200DA81
:1041F000261CAD190B9C0D9E65437243AA189211A3
:104200000BE0C046BC0C0020F802002067467C434F
:104210001C1901340A9D6400625F189E5C00341909
:1042200024890E9F121B3C89121B0F9CA24218DD91
:10423000069D0B242C579C4200DAEB72069E0A2442
:1042400034579C4200DDB372069F09243C578C42D0
:1042500000DA7972069D08242C578C4203DD2972FE
:1042600001E0002A04DD099E964202DA099200E08C
:104270000022846867467C431C1901340C9DA4000D
:1042800062517AE78C466FE70B498268099F069C6A
:10429000056827600C9E4B708A707C2301325B425C
:1042A0009200CB70B218832305200D700B7102F0C1
:1042B0005DFC11B0F0BDC046B8030020F0B5A9B058
:1042C0000FAD059000216422281C04F04BFF06A8C6
:1042D0000021242204F046FF00246300E8580193E3
:1042E00028236343304F02903A1C3232D218049292
:1042F000002605980499835F885FFA215843890056
:10430000FBF726FF029A02361018502E01D00290B9
:10431000EFE73B5F019AC0180234A850322CDCD181
:104320000023E958002901DA0022EA500433642B03
:10433000F7D10024670018206946C0194058192198
:1043400061431A4B01901A1C14328A1802920026FB
:1043500002987200835FA858FA2189005843FBF73E
:10436000F7FE019902360818322E01D00190EFE7CE
:104370000E4B18370233E35E0234C0186B46F85018
:10438000122CD7D1012252420023990006A841588D
:104390008A4202DADAB203920A1C0133092BF4D101
:1043A000039829B0F0BDC046B2910000B299000058
:1043B000F0B585B00192021C5232041C0D1C861C03
:1043C0000292B31E0422A85E03930022AB5E184F34
:1043D000C01A01997843FBF7BBFE039B0199188033
:1043E0000222AB5E0622A85E0435C01A7843FBF7B2
:1043F000AFFE029B308004369E42E2D100230D4A7C
:10440000E15A56329A5A8A1AE2520233502BF6D1A6
:104410000025635FFA2080005843074B2633E95E8E
:10442000FBF796FE60530235502DF2D105B0F0BD7A
:10443000A0860100329B0000B29B000030B5002234
:104440000C7D131C8D5CA54201D00133DBB201321F
:10445000142AF7D1022B14D8012303700B7D0621F7
:10446000181C884301280CD1032B0CD003D8101C36
:10447000012B09D005E01620052B05D01720072BAE
:1044800002D0002000E0152030BD0000014B186074
:104490007047C0469C0C0020014B18687047C0460E
:1044A0009C0C0020014B18607047C046980C0020FF
:1044B000014B18687047C046980C0020014B1860EB
:1044C0007047C046940C0020014B18687047C046E6
:1044D000940C0020014B18687047C046FC00002077
:1044E0008D23013B002B01D0C046FAE7044B10227C
:1044F0001B78DBB21807C00F134018437047C04643
:104500002B0000500F4BF7B518261E700E4BA0273E
:104510001E70FFF7E5FFFF050B4B01AC00252C37A4
:1045200060701D703E70FFF7DBFF064B20703D7022
:104530001D7023786278181C5040400013400343DC
:10454000D8B2FEBD2A0000502D00005010B50D4B12
:1045500000201B78AA2B12D10B4B1C780B4B64B29A
:1045600018780B4B40B219780A4B20181A780A4B6E
:1045700049B21B7840188018C01A43425841C0B253
:1045800010BDC0465000020051000200520002005F
:104590005300020054000200550002008023DB0299
:1045A0000022188059809A80C046024B188880B239
:1045B0007047C04606000400154BC0229200985870
:1045C0001449014099509958FF20814340200143EC
:1045D0009950985810490140802000040143995097
:1045E000985880210002000A0906014399500222CE
:1045F0001A6001221A60082104221A601960FC3333
:1046000000215960054B19690A431A617047C04679
:1046100000E100E0FF00FFFFFFFF00FF00ED00E012
:1046200013B5094A042413780021DBB21C4301911D
:104630000198F421FF31884205DC1370C0461470E4
:1046400001990131F3E713BD0D00005013B50022AD
:104650000192A022D205D06BC021C9000143D163D1
:1046600001AB187803218843012108430C24A0439F
:10467000042420433024A043102420433F2420401E
:1046800040242043187098780F24A0430724204327
:104690009870D8780143D970019B936113BD0000D5
:1046A0000122A023DB051040020603499869084057
:1046B000104398617047C046FFFFFFFE82B00022A2
:1046C000019201301F2201AB1040C9B21870481C82
:1046D000023110400A4092005870DA70019AA0230B
:1046E000DB05DA61196A024A0A401A6202B07047B1
:1046F000FFCFFFFF0002064B000A0138002258607E
:104700009A6005221A60C0461A68D103FCD570472A
:1047100010E000E0F0B5534F85B03B681A1C5432EE
:1047200015780232596D127857331E780F2314070B
:10473000994312092D0701922D0F0B1C80222B4348
:1047400052001343484A0395484D1340484A2B40B2
:1047500048491340240F0B400199220413430A05D2
:1047600045493607360F0B40009613433206434E39
:10477000029433401343424AA024E4051340E3600B
:10478000FFF74EFF3B68E26855331B781540DB06A8
:104790009B0FDB021D43E560E26880239B0013430F
:1047A000E360E26880239B011343E360029C039D66
:1047B000FFF7CCFE002813D0324F882039781E3402
:1047C000C9B2FBF7C5FC39784443C9B28820FBF76E
:1047D000BFFC0F3545431E3C00230F3D9C4203DBCD
:1047E000231E0F2B00DD0F230F22954200DD151C29
:1047F000A024E4051F491A40E36812040B40134348
:10480000E360EB43E268DB171D400F239A431D4032
:104810001543E560E368F022934380221343E3608D
:10482000E368154A18481340E360E3683340E360E7
:10483000FFF760FFE26880235B051343E3600099A4
:10484000E2680B0616401E43E6601048FFF752FF71
:10485000019B09491A05E3680B401343E36005B067
:10486000F0BDC046980C0020FFF9FFFFFFE7FFFFF7
:10487000FFDFFFFFFFFFF0FFFFFF0FFFFFFFFFF076
:10488000FFFFFFEF54000200FF0F0000FF6F00006A
:10489000064A074B1268012094321268197890403A
:1048A000021C0A43D2B21A707047C046FC000020B6
:1048B000290000500549064B09681A7894310968A7
:1048C0000120884082431A707047C046FC000020D7
:1048D00029000050044B1878044B1B6894331B6864
:1048E000184101231840704729000050FC000020A7
:1048F000044B82B0019001AA188092789A7002B09D
:104900007047C0462400005007B500F0DBFD064BA1
:10491000019001AA188092789A70044B00221A70B4
:10492000034B0122DA7707BD24000050800C0020E1
:1049300008000050034B00221A70034B0122DA7763
:104940007047C046800C00200800005072B6084B2B
:104950001B5C002B03D1C04662B630BFF6E762B6DF
:10496000A023DB059968034A0A409A607047C04655
:10497000800C0020FFFFF9FF72B6074B1B5C002B79
:1049800002D1C04662B6F7E762B6A023DB0599689C
:10499000024A0A409A607047800C0020FFFFF9FF2E
:1049A000A023DB055A680121120E58689143034A7F
:1049B000090602400A435A607047C046FFFFFFFEE7
:1049C00008B5074B1B681A1C5C3212785D331B78E4
:1049D0005200013250439940FBF7BAFB08BDC04674
:1049E000980C002008B5044B1B685F331978490008
:1049F0000131FFF7E5FF08BD980C002008B5A023A2
:104A00000120DB055870FFF7A1FFFFF7C9FF08BDC4
:104A1000F7B5A026041CF605042804D1524B1B68E8
:104A2000DF6E1B6F21E0514B1B689F6CDB6C736169
:104A3000FBF75EFDE7300378002B17D004F02CFB6A
:104A400004F092FA01797F22114089040191716981
:104A50000B1C47490B400199194371614179444B43
:104A60000A40716992040B4013437361A023DB0574
:104A70001F611E691F231E40FFF768FD00280AD032
:104A80003C4B882019780436C9B2FBF761FB4643DA
:104A90000023043E03D4331E1F2B00DD1F23A0225E
:104AA000D20510691F210B40884303431361022C78
:104AB00016D007DC002C13D0012C2DD12B4B1D68F8
:104AC0005E3529E0042C07D023DB052C24D1264BAE
:104AD00000241D6877351FE0234B1D6874351BE0EB
:104AE000FBF706FD031CCC331B78002B03D01E4BB9
:104AF0001D68453510E0E7300378002B05D004F041
:104B0000CBFA04F031FA851D06E0184B1D685B35C1
:104B100002E0164B1D686135A023DB055969287832
:104B20003F22104091430143596168781F215D691C
:104B300008401149C0022940014359610F496400EE
:104B400009680C19211C53310878596810409143A9
:104B5000014359605434217858680A401102084AC8
:104B600002400A435A60F7BD9C0C0020980C0020BC
:104B7000FFFF03FE54000200FF07FFFFFC000020C0
:104B8000FFC0FFFF214BF7B51A68214B1B685E334E
:104B90001B785B069B0E0193517E00238D005519F7
:104BA000581E5B18002B25D053181B189B7E8024A1
:104BB000D3185E78A023DB055F68E4033C435C60A8
:104BC000019CB606240400945F68B60EBC46114FE3
:104BD00064462740009C27435F60C0462436760029
:104BE000F65A84002C1966675E680B4C34405C6092
:104BF000031CD5E7537E094974324B700423CB70F4
:104C00000F20B0230B7101F0B1FFF7BDFC000020B5
:104C1000980C0020FFFFC0FFFFFFBFFF0401002032
:104C2000F7B5FFF7AFFF114B00241D686E7E731CB4
:104C30009B005B420093B300EB180193009B043C84
:104C40009C4207D0019B01211F19786FFFF7B8FE26
:104C50007867F3E706492A1C0423CB707432B0232B
:104C60000F204E700B7101F081FFF7BDFC0000209A
:104C700004010020044B00225A70A023DB055A7067
:104C800001221A707047C046800C0020A023DB056B
:104C90009968064A0A40802189020A439A60044AB8
:104CA0000021917001229A707047C046FFFFF9FF02
:104CB000800C0020014B1B68D86E7047FC00002060
:104CC000014B1B68D8667047FC000020A023DB0561
:104CD0009868C0B2704730B5A023DB059B68DBB293
:104CE00083420ED001DA013300E0013BA022D2055D
:104CF0009568FF211C1C8D430C40291C21439160A9
:104D0000EEE730BDA023DB059968802252020A43FA
:104D10009A609968094A0A409A609A6812011209D1
:104D20009A60D968064A0A40DA60D968054A0A409A
:104D3000DA60D968044A0A40DA607047FFFFFFF082
:104D4000FFFEFFFFFFDFFFFFFFFFFFEF1B4B10B575
:104D50001A680121131C52331878A023DB059C68C4
:104D600008401749000421400143996053321078EC
:104D70009C6814490007000921400143996011789B
:104D80009A6809091201090712090A439A60D96849
:104D9000802252000A43DA60D968802292010A43D5
:104DA000DA60D968802252050A43FA20DA6080006E
:104DB00000F0ACFBFFF79EFC10BDC046980C002035
:104DC000FFFFFEFFFFFFFFF008B50020FFF7BEFD6D
:104DD00008BD0000034B1B685C33187840000130AD
:104DE0007047C046980C0020024B1B685D33187852
:104DF0007047C046980C00200048704700100050D3
:104E000000487047002000500048704700400050A4
:104E1000064B1B685879064B02301B6842331B78DF
:104E20005843044B8000C0187047C0469C0C0020BB
:104E3000FC00002004400050F7B5194B051C1C680D
:104E4000A3795E1E10D36279013A0BD36179501CAD
:104E50000231594341181348890009180868E8408D
:104E60000860F1E7331CECE7FFF7D2FFA37A0022DA
:104E700001339C466346013B9C460FD3617A960002
:104E80000191861900230199994205D09F00F1599B
:104E90000133E940F151F6E75218EBE7F7BDC046A0
:104EA0009C0C002000400050064B1B685879064BB4
:104EB00002301B684E331B785843044B8000C018E7
:104EC0007047C0469C0C0020FC00002004400050AD
:104ED000074B1B68DA795879064B02301B680132A0
:104EE00046331B785843044B10188000C018704795
:104EF0009C0C0020FC0000200040005070B53F4B8F
:104F00001D682A7853B2042B18D13D4B19680B1C2D
:104F100076331E7802235D1E6FD34A79013A0BD394
:104F20004879541C023058432018364C8000001930
:104F30000468F4400460F1E72B1CECE7002A45D03C
:104F4000022B21D1FBF7D4FACC3003782C4C002B68
:104F500002D02368473302E02B4B1B685D3318787F
:104F6000FFF76AFF2568EC79002C2FD0FFF7B0FF20
:104F7000061C013C2AD3697A201CFBF73FF9890003
:104F80008A59A300F250F4E7032B03D11E4B1B6890
:104F9000633318E0012B11D1FFF786FF184B061C75
:104FA0001B685C79013C11D32B1922331B789B00C1
:104FB0009859FFF717FDA300F050F3E7052B05D133
:104FC0000F4B1B6879331878FFF736FF0E4B1B68C1
:104FD0005A331B78002B10D0094B1A685379013BC8
:104FE0000BD35079947902306043591C0918054855
:104FF0008900091800200860F1E770BDFC0000205E
:105000009C0C002000400050980C002008B5A02304
:105010000120DB055870FFF799FCFFF7C1FCFFF793
:105020006DFF08BD70B5041C104E114D11D101204B
:10503000FFF7EEFC336801221A70A023DB056C70C9
:105040005C701A70FFF7E2FFFFF7AAFCFFF7E8FDBC
:105050000224201CFFF7DCFC336800221C70A02314
:10506000DB056A705A7001221A7070BDFC000020C6
:10507000800C002008B5FFF7D5FFFFF7C7FF08BD7C
:1050800010B5A023DB051C6A0005064A000D0104CB
:1050900022400A431A621A6A120B12031043186262
:1050A00010BDC046FFFF00F073B5164BA0221B6871
:1050B000D2059168196D503391601C78FFF746FA5C
:1050C000114D002810D0114B114A1B7812782E6810
:1050D00052B25BB20092201C1021D12201F01EFEC0
:1050E0002B6830671B6FE418002C01DA002402E003
:1050F000FF2C00DDFF242B68E0B2DC66FFF7EBFD40
:1051000073BDC046980C0020FC0000205300020034
:105110005200020008B5002801D0012801D100F09A
:1051200041FEFFF7C1FFFFF7F5FAFFF78FFA08BD61
:1051300070B51F4B0D211B68A0B0DA7A00230C3A22
:10514000D2B291425B410321C91AA023DB05586901
:105150003F2210405C688022D20322435A60421EE4
:10516000A023D2B2DB05FF2A11D05E683F25114C87
:1051700015402D0434402C435C60C0460C1C243484
:1051800064001C5B6D465300EC52013AE8E7596835
:10519000094A0A4009495A6002234870CB7003202B
:1051A000B3236A460B7101F0E1FC20B070BDC0462C
:1051B0009C0C0020FFFFC0FFFFFFBFFF0401002089
:1051C000F7B5041C02F0E4F8124B1A68002350688B
:1051D000411C0191019D16689D420CDB97680136C8
:1051E0007E4399008C469E1900216546B6006151A8
:1051F00001333151EEE701239E420ADB956800211D
:105200005D43AF002D180135AD00395101332951EF
:10521000F2E7F7BDF8020020044B054900221A60AE
:1052200059609A6005221A607047C04610E000E09D
:10523000FFFFFF0010B5A023DB059C6899680B4BAE
:10524000C9B21B68E4031B6FE40F591AFF31E62350
:1052500059430134064BA040C918041C0548FAF70D
:1052600077FFC1B2201CFAF773FF10BDFC000020CD
:105270005C5D000040420F00014B00221A60704745
:1052800010E000E013B50B4C0B48A368C01A019363
:10529000FFF7D0FF094901234B7004230190CB7025
:1052A00000206F2301AA0B7101F060FC002301981C
:1052B000236016BD10E000E0FFFFFF0004010020A6
:1052C00010B5041CFFF7A8FF201CFFF7ABFEA023BE
:1052D000DB0501205870FFF74FFBFFF761FBFFF77D
:1052E0000DFEFFF7CFFF10BDF7B5234800F00EF914
:1052F000FFF700FA214F0025214E224CB7421FD262
:105300008036F31B2026832B00DC9E100123667061
:1053100000203A1C211CB610E370207101F026FC1D
:105320003B1C321C013A08D3002D04D116491868E1
:10533000884200D01D1C0433F4E7B600BF19DBE738
:105340000E4904226B1A01270193E270A723211C46
:1053500001AA002067702371843601F007FC042342
:10536000751BE3700020A823211C01AA019567701A
:10537000237101F0FBFBF7BD801A0600C40C00206E
:10538000801B002004010020CDCDCDCD014B1B683A
:10539000587E7047FC00002070B5051CFFF784FDA7
:1053A000094B1C68637E9A00AD180022511ED2186A
:1053B000002A08D0E2185218927E920016588A00ED
:1053C000AE500A1CF2E770BDFC00002030B50A4B5D
:1053D0001B685A7E94001C195300C0180023013327
:1053E000D11A013106D09D00651B59006D6F4942ED
:1053F0004552F4E730BDC046FC000020F8B50C1C57
:10540000051CFFF761F8144908688379013B11D343
:105410000E687279013AF9D30E6870790F4E5843CD
:1054200036688018F6182818603607783679BE195D
:105430000670EFE70B68DB79013B08D3074AE15CB4
:105440001268D218783212798A18E254F4E7281CCC
:10545000211C00F0F9FEF8BD9C0C0020980C0020E7
:10546000134BF7B51C686946E26800AF131C0E3396
:10547000DB08DB00C91A23698D460E33DB08DB002D
:10548000C91A0C4B6D461E688D467960281C311C6C
:1054900003F026FEBA23FF33F1182269786803F07F
:1054A0001FFE281C7968FFF7A9FFBD46F7BDC0465F
:1054B000F8020020940C0020A023DB0518690006E8
:1054C000400F704738B5A023DB0599689D680C4BE9
:1054D000041C1B680B481B6FED03C91AC943E62364
:1054E000C9B25943084BED0FC918FAF731FE054B05
:1054F00001355843211C2841FAF72AFE38BDC04621
:10550000FC00002040420F005C5D000038B5A02385
:10551000DB0599689C680A4B051C1B6809481B6FD2
:10552000E403C91AC943E623C9B25943064BE40F41
:10553000C918FAF70DFE68430134204138BDC04652
:10554000FC00002040420F005C5D000008B5002810
:1055500007D0481006380123132900DC0023C018A7
:1055600006E00B2900DD0E39081C0321FAF7F0FDD7
:1055700008BD0000F0B5C04BA9B01B680025029320
:10558000DB7A071C0C3B281CDBB20D229A426841D7
:10559000BA4B03261B68361A03963E6801934733BD
:1055A0001E70019BC4B278684A3304940DAC291C68
:1055B00018706C22201C03F0D5FDB14B0B951A68B6
:1055C0000C95231C62CA62C323CA23C343CA43C3C4
:1055D000012124234B43221CE31861CA61C361CA21
:1055E00061C361CA61C3039D0131A942F1DB002699
:1055F0000396341C029D6B799C424CDA029D049800
:105600002B19DD7A0BAE291CFFF7A0FF365C242294
:10561000311C5143B446661C06960B180DAEF618A5
:105620000596059B069E1E711F2D08DC0DAE711898
:105630000123CA68AB401D1C1543CD6011E00BAEC1
:10564000335C0DA95A43203D01238A18AB401D1C31
:10565000137E9906890E0D433F210D408B431D4358
:105660001576019D3F23061C2A191E4005966546A6
:105670005678A901059D9E4335431D406346294345
:105680000133039E5170DBB20BAA13549E4200DA21
:1056900003930134AEE7019B039E493300241E703F
:1056A0000294754B029C1B6898798446844200DB07
:1056B000D8E0029D5B191A1DD67F714A12680492C8
:1056C0005A321278059205980022904205D0614620
:1056D00001398D4201DA0533DA7F0123301C191CB0
:1056E00020381C1CB1408440201C06913F210840FA
:1056F000111C20391D1C8B40DBB20993039B242114
:10570000013B4B430790039C28A89540C31808957C
:105710005C3B0194019D002D41D0019D2421013D60
:1057200069430DA8411801957C68CD781F2004407D
:10573000854325430020CD70186018314C783F20F8
:1057400084434C701F2E04DC1968069C21431960A9
:1057500004E04C78079D84432C434C700598002846
:105760001BD06146029C01398C4216DA1F2A04DCE8
:105770001968089D294319600FE0019C24216143A9
:1057800028AD691854394878099C8506AD0E254323
:105790003F242540A04328434870243BBAE7049E99
:1057A000029C331934788033A4065D78A40EFEF78A
:1057B000CDFE002813D0334E882031780135C9B290
:1057C000FAF7C6FC31784543C9B28820FAF7C0FC25
:1057D00002344443013D023C019A6E1C03D02A1E50
:1057E0001F2A00DD1F223F203F2C02DCE043C017B0
:1057F00020400590019C039DAC422CDA019C24259D
:105800006C430DA91F26101C0B19304004905878CA
:10581000B043061C0498064305985E703F2630404E
:105820000490605CB043061C0498064366543968D3
:1058300037291EDC4D4314496D18291C51CB51C129
:1058400070CB70C131CB31C13B68019E0133013651
:105850003B600196CEE7029E7B68013601330296DB
:105860007B601EE7054B3A681B68012048331A70BD
:1058700000E0002029B0F0BD9C0C0020FC000020BE
:10588000980C0020540002000080005030B585B014
:10589000FEF71AFE064B01A81B68021C603332CBD0
:1058A00032C2FFF767FEFFF7DBFD05B030BDC04633
:1058B000FC000020F0B5604B95B01B6800270493F6
:1058C000DB7A051C0C3BDBB20D22381C9A42784176
:1058D000C3B20793594B29681B680BAC01934B3338
:1058E0001970019B6A684E331A70019B391C4D3345
:1058F0001F702422201C03F035FC514B09971B68B4
:105900000A970293029A231C43CA43C343CA43C360
:1059100043CA43C3019E237E77769B06E6689B0EAF
:1059200005960693049E73799F4234DA049E079885
:10593000F319DB7A191C0393FFF708FE09AB1B5C14
:10594000002B0AD1019E717E4A1C72767118FAB240
:105950000BAE8A76013231180A71019EF2190BAE34
:1059600031180979039E22320139117001221F2E4C
:1059700004DCB240059E1643059607E00399069E97
:1059800020398A4032433F210A400692013309AA56
:1059900013540137C6E70BAB059E1A7E0E963F21C6
:1059A000069E02988A43324306781A76B606B60EE9
:1059B000FEF7CCFD00280AD0224B88201978023649
:1059C000C9B2FAF7C5FB46430023023E03D4331E97
:1059D0003F2B00DD3F2362781F2120788A436270CD
:1059E0003F2290431340034323706868E3780840E4
:1059F0008B43617E034391436176296824224A43A5
:105A0000E37000231293139323610F4BD218131CDE
:105A100043CC43C345CC45C346CC46C32B686A68D8
:105A2000013301322B606A60044A012012684C3253
:105A3000137015B0F0BDC0469C0C0020FC00002087
:105A4000980C00205400020000800050F0B5D04BAC
:105A5000A5B01B68002601933B331B78041C0C3B4C
:105A6000301CDBB20D229A427041CA4B03271B68DF
:105A70003F1A0397276802933F331F70029BC5B2FA
:105A800060684233059509AD311C18706C22281CE2
:105A900003F068FBC04B07961B68089624332A1C4A
:105AA000C2CBC2C243CB43C283CB83C201212423D6
:105AB0004B432A1CEB18C1CAC1C3C1CAC1C3C1CA66
:105AC000C1C3039E0131B142F1DB019F0025049760
:105AD0000395019D049F6B7A7E1B9E4243DA049BD3
:105AE00005983B331D78291CFFF730FD07AB2422B6
:105AF0001B5C1F2D09DC5A4309AFBA180123D1687A
:105B0000AB401D1C0D43D5600FE0534309AAD318C9
:105B1000203D0122AA40151C1A7E9106890E0D43D4
:105B20003F210D408A432A431A76029F07AABD19D6
:105B30003835AE783F23115C9E43B446071C8E0176
:105B40001F400096664637431F40009B01311F43AC
:105B5000AF70039DC9B211548D4200DA0391049EC7
:105B600001360496B5E7039E029BF6B24133002747
:105B700004961E700197864B019E1B689A7A964286
:105B800000DBAEE0019D24AF5A19403210780122AB
:105B9000011C2039161C8A403F210A400592039AB5
:105BA0002421013A514386407918039A02965C39C0
:105BB000013A1FD32425554309AE676875191F267E
:105BC00037400097EF78B7433E1C009F3743EF7094
:105BD0003F2618351F2804DC029F0F606F78B743FB
:105BE00005E000270F606F78B743059E37436F705D
:105BF0002439DDE7674A11680022587A824210DAB8
:105C00008818383085782426A806AD097543A7681A
:105C1000800E281809AD0137281807710132A760D6
:105C2000EBE75D4B1B689A1D0533D67FDD7FF606DB
:105C3000AD06F60EAD0EFEF789FC002813D0574FC7
:105C4000882039780136C9B2FAF782FA39784643A2
:105C5000C9B28820FAF77CFA02354543013E023D7D
:105C60000021771C03D0311E1F2900DD1F213F2D8D
:105C700002DD3F20029003E0EB43DB171D4002955D
:105C80000022039FBA4228DA2425554309A81F267B
:105C90000F1C4319374005975F780132B7433E1C0C
:105CA000059F37435F70029F3F26374005972F5C63
:105CB000B7433E1C059F37432F5425682420454396
:105CC000374E7619301CE0CBE0C0E0CBE0C0E0CB33
:105CD000E0C0236801332360D3E7019D01350195BE
:105CE00049E72C4A27681568049E2A1C4032177021
:105CF0002068D07061680532517016700022597AA0
:105D00008A4210DAA9183831897824208E06890948
:105D10004843B60EA168801909AF013138180171E6
:105D20000132A160EBE7002610AF0296029E0398B5
:105D3000864226DA3B1C00210C3B1960029B24267C
:105D4000734309A8C018427E031C01903F20824380
:105D50005A76381C082203F005FA2168104A71436C
:105D60005218131C019A243743CA43C343CA43C37E
:105D700043CA43C32368029E01330136236002965F
:105D8000D4E72368443501202B7025B0F0BDC04610
:105D90009C0C0020FC000020980C00205400020005
:105DA00000800050F0B5674B00241F680D22FB7A7D
:105DB000211C0C3BDBB28BB09A4261410326CBB273
:105DC0000C22761A07A8211C019303F0CBF9059445
:105DD00006947A793D1C02920299EB1B8B4213DAEE
:105DE000E97A0198FFF7B2FB072801D90020A6E065
:105DF00005AA135C0135B342F8DA0133DBB2135460
:105E00009C42E9DA1C1CE7E701220792B8790021DD
:105E100081420ADA131C9D1AA54203DA372BE5DC0E
:105E20000133F8E701311A1CF2E70792FB79002BE6
:105E300011D1002307A80793FFF73CFD07A8FFF740
:105E400099FB404B404D1B68DE79002E3BD007A8E4
:105E5000FFF7FCFD4DE03B1C3B331B7800250C3B62
:105E6000DBB20D22291C9A426941CAB20292032276
:105E7000521A0192059506957B7A3E1C0393039A6C
:105E8000F31B934214DA331C3B3319780298FFF763
:105E90005DFB0728AAD805AA135C019901368B423D
:105EA000A4DA0133DBB213549D42E8DA1D1CE6E7A5
:105EB000EB43DB171D40BB7A5D43079B6D00ED187C
:105EC000372DB6DD92E72868311C04223F3003F0FD
:105ED00049F92868311C0422433003F043F92B6848
:105EE0000799CAB2191C3F3144330A704A700A71CB
:105EF0001A702D6864002B1C4B331A78073BDA7339
:105F0000291C1B7854310B704A70083909782A1CF7
:105F1000563211700F3A1678291C5731281C0E7012
:105F200059305374022203F0DBF82B1C5B33341915
:105F30001E705C702E66113B1B7801206B660BB0E7
:105F4000F0BDC0469C0C0020FC000020F0B5B94B11
:105F5000B94A1B6812681C6EABB006940192D27AE3
:105F600000250C3A2E1CD2B20D2191426E41F7B29F
:105F70001A1C04974F320327147052330FACBF1B07
:105F80000126291C1E706C22201C03F0EBF8019BDB
:105F90000D950E954833221C23CB23C223CB23C25D
:105FA00023CB23C224237343221CE31823CA23C315
:105FB00023CA23C3013623CA23C3BE42F2DB019E98
:105FC000002776793C1C03960297039EB4423ADA86
:105FD000019D04982B19DD7A291CFFF7B7FA0DAB48
:105FE0001E5C2422311C5143B446661C05960F18D2
:105FF0000FAEF719059E3E711F2D08DC0FAF791803
:106000000123CA68AB401D1C1543CD6010E01B5C2A
:10601000203D5A430FAB9A180123AB401D1C137E41
:106020009906890E0D433F210D408B431D43157684
:1060300063460133029DDBB20DAA13549D4200DA80
:1060400002930134C1E7069F012404970194029C46
:106050002422013C62432AADAA18029B08945C3AB0
:10606000013B13D32420584300250FAE1560301890
:10607000467E3F24A64346765560857EC178A5437B
:10608000402421438576C170243AE9E76A4B019C9C
:106090001F68013CB879BC4607900994231C099EEF
:1060A000079F9A1BBA4256DA019D0122511B614497
:1060B000281CC9180138C0B2233109780B90581038
:1060C00010400A90081C2038161C8240D2B2089F4B
:1060D000059224227A432AA88E408218029F0396B2
:1060E000583A013F35D3242078430FAC2018C678A6
:1060F000019D1F242540A6432E430B9DC6700A9E7A
:106100006CB2B44212D01F2905DC101F0468039D35
:106110002C4304601BE0447E059DA606B60E2E436C
:106120003F252E40AC433443447610E01F2904DC65
:106130001068039E3043106009E0847E059DA6062A
:10614000B60E2E433F252E40AC4334438476243A8A
:10615000C7E70133A3E7394B1B68DB1980335E784F
:10616000634648331D78AD06AD0EFEF7EFF9002803
:1061700013D0334C882021780136C9B2F9F7E8FFF3
:1061800021784643C9B28820F9F7E2FF023545433A
:10619000013E023D0024701C03D0341E1F2C00DD84
:1061A0001F243F2D02DD3F21039103E0EB43DB176A
:1061B0001D400395049D24236B43224E00219B190F
:1061C000029DA94221DA24254D430FA81F26271C32
:1061D00042193740059757780131B7433E1C059F58
:1061E00037435770039F3F26374005972F5CB743CF
:1061F0003E1C059F37432F54181CE0CAE0C0E0CA7C
:10620000E0C02433E0CAE0C0DAE7EB43049E019F1C
:10621000DB172B40F618013704960197032F00D0A7
:1062200015E7044A069E1268F118CB185032137015
:106230002BB0F0BDFC0000209C0C0020980C00202E
:106240005400020000800050F0B5364B85B01B684A
:1062500002901A1C03913F321578334A00201168CE
:10626000041C8A7A94422ADA021C4F7A161ABE4219
:106270001EDA9E193836B678B7090096EF1924262B
:106280007E432A4FB4463E1C009F66440196BE06DC
:10629000039FB60EB446BE5C3F2E00DD3F26F6B22D
:1062A0000096019E0132371C009E67443E77DCE772
:1062B000181C4130007801342D18101CD1E71A1C2D
:1062C0004732147800208A79904228DA00224D79EA
:1062D0000195AA421DDA9E187678B709E719039747
:1062E00024273D1C039FB6067D43AC460F4DB60EDA
:1062F0002F1C019D674445430397029FBF187D5D96
:106300003F2D00DD3F25039FEDB2BE1935770132E9
:10631000DDE71A1C493212780130A418D3E705B022
:10632000F0BDC046FC0000209C0C00200080005006
:1063300030B50F4B1B689979884203DA1B18043378
:10634000D87F14E05A798D18411AA84202DA5B18F6
:10635000D87A0CE09C7A8A1A2D19A84203DA9B1885
:106360004033187803E0141B1B193833D87830BD3C
:106370009C0C0020F0B5D34DA024E405A3682B6845
:1063800097B059799A7900AF8A18597A9B7A52183E
:10639000D3181A1C5A433B62D31DDB08DB00684646
:1063A000C01A85466B46FF213B6102F0DBFEFF20F1
:1063B000FFF7ACF8C44B69461B1A386A7B60C00013
:1063C000031C0E33DB08DB00F860C91A386A8D46FF
:1063D0006B468000FB61031C0A33DB08DB00C91A33
:1063E000002200233A637B63B860B961E268B74B6F
:1063F0008D461340E3602B685C79B24B013C1B680F
:10640000621C14D01B19381CD97A5030202202F09B
:1064100049FE3D6D58207A6DAB00C019C3180121AB
:10642000283B91400A1C19680A431A60E5E79C79E9
:10643000A44B013C1B68621C15D01B190433381C8B
:10644000D97F5030202202F02DFE3D6D58207A6D0C
:10645000AB00C019C3180121283B91400A1C1968E0
:106460000A431A60E4E75C7A964B013C1B68621CA5
:1064700015D01B193833381CD9785030202202F03F
:1064800011FE3D6D58207A6DAB00C019C318012173
:10649000283B91400A1C19680A431A60E4E79C7A79
:1064A000013C621C17D0874B381C1B6850301B19ED
:1064B00040331978202202F0F5FD3D6D58207A6DA9
:1064C000AB00C019C3180121283B91400A1C196870
:1064D0000A431A60E4E73D697D610025FD62FD6ABB
:1064E000386A854200DBDBE00021FA68F86902F0D7
:1064F00039FEA0240021BA68B86902F033FEE40531
:1065000000232363636B3F26B34363633D6BA56343
:10651000786BC0B2B86230407862E36BB343034338
:10652000E3636420FEF7F2FFFEF7E4F8F86AFFF792
:10653000FFFEC1B2381C4830202202F0B3FD396B97
:106540007A6BFB6CB963FA63BA6C012199405820ED
:106550000B1CC01991004118081C203802689A438E
:106560000260B86C131C002808D028390A68534010
:10657000626B3340B2431343636301E06B402363B8
:10658000A024E405A563E36B796A3F26B3430B437C
:10659000E3630A20FEF7BAFFFEF7ACF8E26B802354
:1065A0005B001343E363BA6B5540A563FB6BBA6AA8
:1065B0005A40E36B3240B3431343E363FEF72CFED0
:1065C000FD6BBE6BFB69AC460124414A7D68916856
:1065D000A94214DB3F4A65461068526830402A40A1
:1065E0005D68954203D3F0D11D688542EDD2BD6947
:1065F000DA60A2009860A95001340833E5E7FEF79D
:106600003BFEA023DB05D96B334A0A40DA63012C39
:106610003ED0651EF869ED004519013C002C37D0CD
:106620002B1C083B1A6829685B6891436A683E6ABC
:106630009A43A30039647A64013EBB62FA6A9642C7
:1066400024D0301CFFF774FE011C381C503020226F
:1066500002F028FD7B6D0122386D9A405821131CF1
:10666000C91982008A18183A12681A420CD0BB6AFB
:10667000BA691720D25840425043184BC018FEF751
:10668000D9FD796900118855013ED7E7083DC4E777
:10669000FD6A386A0135FD627D692D187D611EE74E
:1066A000C3B2381C50300370437083700023C37032
:1066B000037139690123437100F09CF9BD4617B09D
:1066C000F0BDC0469C0C0020FFFFFF00FFFF0FFF46
:1066D00010E000E040000050FFFEFFFFE9FFFF1662
:1066E000014B18607047C046A40C0020014B186095
:1066F0007047C046A00C0020F8B5F9F7E7FE071C6C
:1067000000F046FE061CFDF7C7FE2D4D1022041CAE
:10671000391C286802F0E4FC32882B681A74120ACB
:106720005A74B2889A74120ADA74264A12680532C8
:10673000D27F002A03D0A2791A75627902E06279C9
:106740001A75A2795A75E2791F4C9A75231C083381
:10675000AB601E4B6C606E691B783370FDF7D2FE28
:10676000627E217E12020A43A17EF07109040A436F
:10677000E17EEB6809060A43110A1A705970110C80
:10678000120EDA70627F9970217F12020A43A17F94
:1067900009040A43E17F09060A43110A1A71597173
:1067A000110C120EDA71221C2C322D3499711178D1
:1067B000227812020A431A72120A5A72F8BDC046AF
:1067C00014010020F8020020D0BF00004700005054
:1067D000F7B5F9F77BFE051C00F0DAFDFDF75CFE6E
:1067E000144CAA6BE369A56A59685A6002F09CFBD5
:1067F0006860FFF781FF104B226B1B680F481988F8
:106800006D460B0A11715371C0C8C0C589006B4633
:10681000CB589371231C3C3301225A7000229A708A
:1068200002F07CFB064B5860064B1A78236C1A70FA
:10683000F7BDC04614010020A40C0020289C0000D5
:10684000C80300204600005008B5084AD1694B78BB
:106850000749DBB20B72012B05D0022B05D19369DE
:1068600001225A7001E0FEF713F808BD1401002060
:10687000C8030020094B10B51B7A094C012B05D029
:10688000022B05D1A2690023537001E0FEF712F834
:10689000636B7F211A788A431A7010BDC8030020E9
:1068A00014010020F8B5194D0024194E337A012B3C
:1068B00007D0002B18D0022B17D1164B9B695C78A0
:1068C00013E0FEF707F8041C002D0BD1FDF7F2FFD3
:1068D0002E23FF33013B002B01D0C046FAE7FDF722
:1068E000D7FF0A4D013D00E01C1C0A4FFA6953789E
:1068F000327A9A4206D0FFF7BDFFFB69044A5B7803
:10690000137201E0002CD0D1F8BDC046FF2C01006D
:10691000C803002014010020024BDB691878C0B2C4
:106920007047C04614010020024BDB695878C0B2A2
:106930007047C04614010020024BDB699878C0B252
:106940007047C04614010020014BDB699870704706
:1069500014010020024BDB69D878C0B27047C046F2
:1069600014010020014BDB695868704714010020B6
:10697000024BDB69187AC0B27047C0461401002090
:10698000024BDB69587AC0B27047C0461401002040
:10699000024BDB69D87AC0B27047C04614010020B0
:1069A000024BDB69987AC0B27047C04614010020E0
:1069B000024BDB69587BC0B27047C046140100200F
:1069C000024BDB69187CC0B27047C046140100203E
:1069D000034BA0229B691A701A78A02AFCD070473A
:1069E00014010020024B9B6C1878C0B27047C0465F
:1069F000140100200E4B30B59A6CFF2414700D4C1E
:106A0000D864216005788478996A6C430579407967
:106A100064194006400E604308609869A021017027
:106A2000D9691378FF2B02D10B78022BF9D030BD36
:106A300014010020C8030020014B1B681888704710
:106A4000A40C002008B5FFF72DFF024B0022DA60EE
:106A500008BDC046C803002070B5074B074C1A6B31
:106A6000E668011C9579986B2A1C8019751902F04B
:106A700037FBE56070BDC04614010020C80300204C
:106A800008B5074BDB68002B09D0064ADBB2506B18
:106A90007F21194001703C329370FFF7D5FE08BD8D
:106AA000C803002014010020F8B5071C0E1CFFF7D6
:106AB000F9FE0D4C8020636B40421978F6B2084312
:106AC0007F22C0B29043311C1140021C0A43A56BC7
:106AD000A7631A70231C3C339E70FFF7B5FEFFF7C7
:106AE000E1FEA563F8BDC04614010020014B5B6DBB
:106AF000187070471401002073B56C46E271194A92
:106B00000734556D2E7886422AD1FF2028701366EF
:106B1000131C94331B6820789B6880009165D465B2
:106B20001871114B06980C7818608878936A604346
:106B30000C79497900194906490E41431960916958
:106B4000A0230B70516DD3690A78FF2A02D11A78FD
:106B5000002AF9D00A78FF2A02D11A780A2AF3D03B
:106B600073BDC04614010020C803002070B5144C4A
:106B7000636B1D79EDB2012D21D1854058781E78C7
:106B8000000230439E7836043043DE7836063043C8
:106B9000284214D0FF2018710A48A16302608C7843
:106BA0000D78C9786C434906490E074A6143906ADB
:106BB00092690160772111701A79FF2AFCD070BDAB
:106BC00094010020C803002014010020014BDB6B5E
:106BD0001878704794010020014BDB6B18707047E8
:106BE00094010020014BDB6B587870479401002022
:106BF000014BDB6B5870704794010020014BDB6B3D
:106C00009878704794010020014BDB6B98707047B7
:106C100094010020014BDB6B187970479401002030
:106C2000024BDB689872000AD8727047140100208A
:106C3000024B5B691872000A5872704714010020F9
:106C4000024B5B699872000AD872704714010020E9
:106C5000002303600B60204BF7B59A423ADC131215
:106C60001E4C122B25D89B00E418646E002C31D0EA
:106C7000E368013B5D1C2DD0D5B2019565681E1CF3
:106C8000EF5C019D013BED1BF4D42768B300DB5999
:106C9000002B1FD0A268925D521B0A60002A02DD01
:106CA0005D19056016E00E4B403303605B780B60A6
:106CB00010E0E36A666A013B0CD35D00755B551B0F
:106CC000F9D4266A9B00F25852190260A26AD3587E
:106CD0005D1B0D60F7BDC046FFEF000014010020F2
:106CE00094010020C02208B5D2000B4B904206D17F
:106CF0009B691A78052A0DD005221A700AE05B6B91
:106D000084221B7892005B065B0E9B18984201D18F
:106D1000FFF7B0FD08BDC0461401002038B5051CC2
:106D20001C1C181C8D4209DB0498954206DAC01A17
:106D30006D1A6843511AF9F70BFA201838BDF8B5E7
:106D400001254E1E6C00B54202DA165FB0420CDA25
:106D5000A61E1D5F115F9B5F401AEB1A5843935F9D
:106D6000C91AF9F7F5F94019F8BD0135E9E700004E
:106D7000014B18607047C046B00C0020014B1868EA
:106D80007047C046B00C0020014B18607047C046E9
:106D9000A80C0020014B18687047C046A80C0020C2
:106DA000014B18607047C046AC0C0020014B1868BE
:106DB0007047C046FC020020F0B5041C87B00020DC
:106DC0000D1C2C4902920393021C4F230B71FFF7F9
:106DD000CDFE294B00201A685368013B0FD3990060
:106DE0006F5811684E1EB446F7D396687143591810
:106DF000013189000959C91B40186146F2E7D16881
:106E0000F9F7A6F91D4B071C1D681D4C6E88002E56
:106E100003D1236840229A600CE0A9882268701A86
:106E20008001791A0192F9F793F96E2800DD6E203E
:106E3000019B9860AB7964225343029A5343039AAF
:106E400013412A78002A03D02268926853439B1189
:106E500022680C49D36002234B707C235B42CB70C9
:106E60000020502304AA049605970B71FFF77EFEBD
:106E700007B0F0BDBF030020F8020020A80C0020DE
:106E8000FC02002004010020F0B585B001912449E6
:106E9000D2690968051CC9798A40002A00DC0122F0
:106EA00020490968C868191C5043F9F751F91E4B6D
:106EB00002901C6820680390021C571E1AD3636856
:106EC000191C7943C918890069180439013B0FD38B
:106ED000A66801205643B4469C44844466468640D6
:106EE0000198305E029E46430868801B0860ECE70C
:106EF0003A1CE2E70D4E1023B371039B042033705C
:106F00002379311C7370B3702A1C6023F0703371C5
:106F1000FFF72CFE00230120B37105B0F0BDC04681
:106F2000A80C0020FC020020F8020020B80300207A
:106F3000F8B5144B051C1B680E1CD868111CF9F71A
:106F400007F9114B1B681A6994002C19131C043C97
:106F5000013B06D35900715E27684143791A2160CD
:106F6000F5E70A4C1023A3716270042061232A1CE8
:106F7000211CE0702371FFF7F9FD00230120A371AC
:106F8000F8BDC046FC020020F802002004010020E9
:106F9000F0B585B003931A4B00901C6802912568E8
:106FA00001926F1E1BD3636800981E1C7E43F61867
:106FB000B6008619043E013B0FD3A1680122694344
:106FC0008C469C4494446046019980004258306845
:106FD0009446844461463160ECE73D1CE1E7226958
:106FE000039D029C9300E118E8180023043B013A3A
:106FF00004D3CE58C5587419CC50F7E705B0F0BD8E
:10700000F8020020F8B5061C58780D1C4000917855
:107010000130884051789B784900013199408003C4
:10702000F9F796F81349041C0020B423021C0B71D5
:10703000FFF79CFD104B18680268013A0DD34368B6
:10704000191C5143C918890071180439013BF4D344
:107050000F68BF0B67430F60F7E703699900691872
:107060000439013B04D30868820B62430A60F7E7E6
:10707000F8BDC046BF030020F8020020F0B5284B41
:1070800089B01E68274B04921A6803910592264A1C
:107090003168126807900692244A01911768019B93
:1070A000013B01931FD37468019B21496343651819
:1070B000ED18079AAD0002935519013CEFD30499DE
:1070C0002868F8F7F7FF05990B78002B07D0069A88
:1070D000029953181B5DBA685843504300130004CB
:1070E0002860043DE9E70F490F4B34691F680E68BB
:1070F000013C12D3039AA50050590499F8F7DAFF1E
:107100003378002B05D03B19BA33FF331B78584333
:107110008011039B00045851EAE709B0F0BDC04656
:10712000F8020020A80C0020AC0C0020FC0200207B
:10713000FFFFFF3FF0B55C4E89B0336804910792C2
:107140005A499A69049F4A709A68041C8A7058695F
:107150000132042392000870CB700220A023BA18D9
:107160000B71FFF703FD306845690095009E836948
:10717000013E039632D303991A1C59436A43079F71
:1071800094468E00BF196646D218059777005200C4
:107190007F424900A21806978C46023A013B1AD357
:1071A000059F9E00BE598768310C009E7743DF190A
:1071B000049E0137BF00BF596646C91B069F019157
:1071C000BF18391C019F8F53F9177E1817884E403E
:1071D000F6191680E1E7039A0092C7E73349DBB25C
:1071E0004B708B707E236A1C5B420A70CB70221C32
:1071F000A12301200B71FFF7B9FC2D4B00261A6863
:10720000294B166019682B4B8F691B6804970393F1
:10721000FF253B1C013B13D304984F694743FF18DC
:107220007F00E75F039800788742F3DB9E4200DA35
:10723000DEB29D4200DDDDB21068C7191760E9E7D4
:107240001D4901270423CB70381C64230B714F7038
:10725000FFF78CFC164B00201A68164B12681B684F
:107260005B789A421DD910490B6869B29A695B69CB
:107270005A4373B25B1AD90FCB183B41EB18DBB200
:107280009B18AD18BB40BD40295FE35E381C994296
:1072900007DDB218BA40125FD917D00F93424841A8
:1072A000C0B209B0F0BDC046F8020020B80300200B
:1072B000FC020020B00C0020040100202D4BF0B592
:1072C0001D682D4B89B01C680490A7690E1C2868A6
:1072D000391C0392F8F7EEFE284B1B68DB799840C7
:1072E000002800DC0120EB6803995843F8F730FFD1
:1072F00084466069BB005B42421E391C03935143C4
:107300007B005D425343049CC9198900F31861183E
:107310000595069301900024019D013D019515D32B
:10732000069E0A1CA61907963B1C043A013B08D38B
:10733000079D5E00AD5F66466E431568AD1B156028
:10734000F3E7039E059B8919E418E5E70C4C10232D
:10735000A371FBB220706370A37004206023211C12
:10736000049A2371E070FFF701FC0023A37109B0B8
:10737000F0BDC046FC020020F8020020A80C00204E
:10738000B8030020014B18607047C046B80C0020BD
:10739000014B18687047C046B80C002010B5064C69
:1073A0002060808CFFF744FC23683C331878FFF79B
:1073B00047FC01F0F1FA10BDB40C0020014B186835
:1073C0007047C04600030020F7B5444C00212068F8
:1073D0000A22283001F0C6FE206800210A2232303D
:1073E00001F0C0FE2068002128223C3001F0BAFEE6
:1073F000206800210A22643001F0B4FE20680021D8
:107400000A226E3001F0AEFE206800210A22783098
:1074100001F0A8FE206800210522823001F0A2FEC2
:10742000206800210522873001F09CFE20680021A1
:10743000B822A83001F096FE294B24681D68EA693D
:10744000296A5000401A00024900F8F781FE6B6A71
:10745000A96A071CA0605800401A00024900F8F70A
:1074600077FE204BE0601B687F0059681E68013979
:10747000013E0902400036028619791800966661BD
:10748000216105332A1CDB7F271CD832261C90374C
:1074900001929436D635002B06D010880004F8F7F8
:1074A00057FE3860288806E028880004F8F750FE68
:1074B000019B3860188800990004F8F749FE0A4BD0
:1074C00030601B6864211A1C4E32343312781878ED
:1074D000FC345043F8F73CFEE065F7BD00030020A4
:1074E000B80C0020F8020020B40C00200D4B002145
:1074F0001A6830B5131CA03319600B4B1B681B7C3A
:10750000013BDBB2FF2B0BD059000C5A191C343154
:10751000490025B25118002D00DC0024CC80EFE793
:1075200030BDC04600030020F802002010B5022440
:107530008B7804575AB2944200DD8370CB780324D1
:1075400004575AB2944200DAC3700B7800240457EF
:107550005AB2944200DD03704B78012141565AB271
:10756000914200DA437010BDF0B58BB00592059CD6
:10757000069301322301C418089209912589069EB9
:107580002FB20295350145192E892368049636B22B
:10759000B819079028687B4370430799C018F8F71B
:1075A000D7FD696863684E437B4300B2079920604A
:1075B000F018F8F7CDFD00B26060201C109904228D
:1075C0000A3001F08DFD049E029FF31923810023F0
:1075D0002B81069F059D099EAD00BA00AC46331C69
:1075E000B118634408880027DE5F05B2AE4204DAB2
:1075F0001880C878D870897899708449069B096882
:107600000133C86A012583420ADA129E9D40311C6B
:10761000B75861440E683D4035430D600133F1E7D2
:10762000129F0023BB50069E059F291CB140BD4000
:10763000129A0295CE43069FBB421ADA10680142A5
:1076400014D0059DAB4203DA029F384310600AE074
:10765000059DAB4207DD129F381C60440568012779
:107660009F402F43076010683040106001330432A0
:10767000E1E7109D2D786DB20295109D0123EB5628
:10768000029E9E4200DD9BE0109EB67876B2039685
:10769000109E0322029BB256039F0133974200DDE6
:1076A0008CE05A4A039D1168119E8F68C96A7B431A
:1076B00001335B19F61832780497013AB446079102
:1076C000531A012B76DD0121052349420020013B9D
:1076D000002B29D04E4F0126FD187642AE57029D51
:1076E000FF18AE19049D01367543FF790995119E67
:1076F000039D7FB200977719099D7E19009FF619A7
:107700007578013DE3D3079EB542E0DA059FBD429F
:1077100002D0069EB542DAD14F1C03D0A942D6D082
:107720000120D4E7291CD2E7002843D0122A3FD1F8
:10773000089D604605700527013F002F3AD0344B65
:107740000721DA19131C5156012252429A562F4B27
:10775000029D1868AA188068531C4343039E013396
:107760007118119E5B18F0180578002DE4D1139D57
:107770005B005B5B002BDFD012250570258920683C
:107780002EB2594370430902401861685A435D198B
:107790004E43ADB225812DB21202291CB618F8F75E
:1077A000D7FC291C2060301CF8F7D2FC6060C3E7CE
:1077B00063461A70039D0135039569E702935CE700
:1077C0000022AA56109C0123E3569A421BDC109F0C
:1077D0000223FB56109F03203856511C834210DCB5
:1077E0000A48119C0068069D806841430131C91810
:1077F000611808780138A84201D1089E0E70013343
:10780000E8E70A1CDEE70BB0F0BDC046F802002036
:10781000309C0000F0B5A7B02C9C179100940C92FE
:1078200013930A90FCF7E6F8C44B1A68131C9C33B8
:107830001968C34B012908D198321268012A04DD66
:107840001B689D881495DB8803E01B681E881496CE
:107850005B881593BB4B1B68DB6A013B0693069B59
:10786000069E013B002E00D170E1139F9A00069CFA
:10787000D2590894E2400E9206930E9C002CEED052
:10788000B04B089D1B68DB6A9D42E8DA0E9D012221
:10789000154200D14BE1069E0A9F3501089E7D19D5
:1078A00034013C1920682F686E68391A6768F31B29
:1078B000CF17CE197E40DF170F96DE197E400F9F3F
:1078C0000B96B74202DD1092180203E00026080270
:1078D0001096191CF8F73CFC1CAE211C04221290D7
:1078E0000A31301C01F0FCFB291C0A31301CFFF767
:1078F0001DFE286820900821675E07972768079B70
:10790000099708216F5E5843099B079A7B43BA1871
:10791000111CC0180D92F8F71BFC2190099864689F
:1079200022906868079D3B1C6343239068430D9930
:10793000C018F8F70DFC0027249000211DA80C2288
:10794000259401F00FFCF7570124099734570225BD
:10795000189475577B4B1995F6781B6876B21A9672
:107960000D93099E189FBE4200DDA0E0099E199F5D
:10797000360216960797099B079C1A9D0133AC4265
:1079800000DD92E00D98079C80680C9E4343013314
:107990001D190D9F735DF96A013B11908B4246DB07
:1079A0000024012005224042A446013A002A2DD09D
:1079B000654EB718013F3F78099E7FB2F719119EB7
:1079C000013777430597604FBE18F679079F76B267
:1079D00004960C9EF619059FF619049FF6191B963E
:1079E0007678013EE1D38E42DFDA069FBE4202D0B6
:1079F000089FBE4206D1471C06D0B042D5D0012612
:107A0000B446D2E70124D0E7301CCEE7013049D09C
:107A100067466A00002F01D1002C02D12C9CA05A8D
:107A200010E02C9D591AA85AF8F792FB0AE0002B97
:107A300038DB069EB34202D0089FBB4232D12C9C59
:107A40006B00185B00282DD0079D03232902013B02
:107A500028D3109F20AC23AA9E00002F09D095594F
:107A6000169FA2597D1B129F7D432D12551B6D1A27
:107A700008E0A559129C4D1B654392592D12169E84
:107A8000551BAD1BEF17ED197D40FF2DDFDC802668
:107A90007600751B45439C001DAAA6582D1275192A
:107AA000A550D4E7079F013764E7099359E71F9B67
:107AB0001D9C9C4200DD1C1C109D002D06D10B9EC0
:107AC0002B1C002E0DD00F9F0F960B970B9D0F991F
:107AD000A801F8F73DFB3F2800DD3F201A4B18189E
:107AE000037C2D21149E159FC81A70437B43C01838
:107AF000F8F72EFB44431E9BA412A34217DD089CFB
:107B0000069DAC4201DB089506940C9E139F2C9CAD
:107B10001CAB00930196069B029703940A98179951
:107B2000089AFFF721FD069B089D08930695089E7D
:107B30000E9F01367F0808960E979EE600030020F0
:107B4000B40C0020F8020020309C0000274E069F55
:107B500033680121181C98331F60254B18301B68AF
:107B60004942DA6A01F0FEFA069D371C2C1C204BB4
:107B70001B68DA6A944226DA0A98260186190821D7
:107B8000735E002B1CDD3B681A1C983211681B19B0
:107B9000013111601D76A54210D00A9A33687168D0
:107BA00028011018416003603389311C03810A31B8
:107BB0000A30042201F094FA002333810135EDB23A
:107BC0000134E4B2D3E70B499A680C9E1C685D68E7
:107BD0008A7001230132CB70B218302306200C705A
:107BE0004D700B71FEF7C2FF27B0F0BD00030020FF
:107BF000F8020020B8030020C31770B5C4185C4019
:107C0000CB17CD185D40AC4202DB231C2C1C1D1C85
:107C1000A001291CF8F79CFA094E3018037C281C97
:107C2000002B0BD05A22D21A52365200955B5B00C1
:107C300068439D5B00146C432414001970BDC0465A
:107C4000309C0000164BC2171B68801850401A1C4D
:107C5000903270B594331468CA1789181D68514062
:107C600044434D4324142D14AC4202DB231C2C1C32
:107C70001D1CA001291CF8F76BFA0A4E3018037C72
:107C8000281C002B0BD05A22D21A52365200955B78
:107C90005B0068439D5B00146C432414001970BDA5
:107CA00000030020309C0000F0B58DB000AF7B6079
:107CB0007E4BFA601D683961EA6A6946D31DDB08AC
:107CC000DB00C91A8D466C467C625400231C0833C5
:107CD000DB08DB00C91A8D4639620121B8614942CF
:107CE000786A01F03FFA386AFF21221C01F03AFA63
:107CF0006F4B00261B68FB612C6AA64257DAFC68B2
:107D0000F300E31804215B5E002B4DD0331CFC69AB
:107D10000E339B00E3185A68231CFC335B6E520041
:107D2000D318FB62231C98331B687C68BB60B300CC
:107D3000E318002101247B616442B962BB6AB9681F
:107D40008B421DDABA6AB9691301CB1808215A5E51
:107D5000002A10D07A6919680020105E081A796923
:107D600002228A5E5968891AFFF76CFFFA6A90420C
:107D700001DABC6AF862BB6A0133DBB2BB62DDE7E1
:107D8000621C11D07B6A1A576300013207D0396A2E
:107D9000CB181A88F96A8A4206D9198002E0FA6A71
:107DA000396ACA527B6A1E55731CDEB2A4E70024EE
:107DB0003F4B1B68BB6298331B689C4222DA796A8E
:107DC0000E5D73B201331AD0F6B20E207043BB6958
:107DD0003A692101591810184B680A6843800280DB
:107DE0000B89042283800A31083001F079F93A6A5C
:107DF0000E36B96A6300B6009B5A8E19736001345F
:107E0000E4B2D5E70024B86A98300668B44232DAA2
:107E10007E6A335701332BD1BE69210171180822C4
:107E20008B5E002B24D02B6A9C46002363451FDA0F
:107E3000FE68D80030180422805E002815D10E207C
:107E400058433E6930180422865E002E0DD17E6AAA
:107E500033550A684B68028043800B890422838073
:107E60000A31083001F03CF902E00133DBB2DDE712
:107E70000134E4B2C7E70023EC6A2A6AA3420DDAB0
:107E8000BC6AE1180C7E944203DA7A6A145D0C76BF
:107E900001E0FF220A760133DBB2EDE7964200DD16
:107EA000161CBD4606600DB0F0BDC046F8020020AD
:107EB00000030020F0B595B0041C09910A92FFF769
:107EC0007DFA744B0B901B681B6A013B0493049D65
:107ED0000E236B43E418271D049C013400D1D6E027
:107EE0000026BB5F002B00DCCCE06A4B0621186843
:107EF000694B07227956BA561B6800248C460C92AF
:107F00000E93059406940C9EB44566DC05257D57BA
:107F1000664604223602BA560D950F960D9D6346AD
:107F20000133AA4257DC8468511C08916143099DC2
:107F3000C9186B5CC66AB34224DD0523013B002BE4
:107F40002FD0564DEE18ED18013D2D78F6796DB213
:107F500055190135654376B20295099D03962E1C8D
:107F6000039D664475190796029EAE197578002D1B
:107F7000E4D00E9E6DB27519ED7D049E6DB2B542D2
:107F8000DCD109E0002B0BDD0B9D1724EB181C57EF
:107F9000049E0023B44204D10A9C49000B5B00E01C
:107FA0000023391F0025495F0F9E069D891BCC17B2
:107FB0000919614059436D18B91E0026895F1202E4
:107FC0008A1AD11752184A405343059C0695E41863
:107FD0000594089AA2E79C4695E73B1F1A78BB1EBA
:107FE0001B78802A02DD802149008A1A802B02DD5D
:107FF00080214900CB1AD618294B301C1B681A1C4B
:10800000EC3205331168FF330432FEF798FE254B3E
:10801000041C1B680021785E2422995E9A6B402321
:108020001B1B00930023FEF779FE2318059C06987E
:108030005C43059400257C5F5843A501291CF8F793
:1080400087F8291C06900598F8F782F8011C069815
:10805000FFF7F8FD14497880CA7880B212907F202B
:10806000824304234B701343802252421343049DE6
:10807000CB701220B02310AA1095119613940B7197
:10808000FEF774FD049E0E3F013E049624E715B0F2
:10809000F0BDC046F802002000030020309C000024
:1080A000B80C0020B40C002004010020594BF0B59E
:1080B0001B6885B05A681D6A013A120202920E24AA
:1080C0001A686B1E5C43013A1202041900270190E2
:1080D000039204340097002D00D181E04E4F3B689D
:1080E0001A1C50321678012E16D102320020215E61
:1080F000128891420EDD543362881B789A4209D966
:1081000046492672B5230E2000220B71FEF72EFD84
:10811000009601E0002323723E68331C55331B7820
:10812000012B5AD1331C58330021625E1B889A42BE
:1081300053DD231F0027DA5FFF2A0ADDA31E00207C
:108140001B5EFF2B05DD029FBA4202DC039FBB4290
:1081500043DA304B07271B68E7570533DA7F0520E2
:108160000421BC4606272E4B20566156E757002AAD
:108170000ED01A68411A131C94331B6809024B4332
:1081800060469032C71B11683F021B1479430DE013
:108190001A686346DF1B131C90331B689432411A24
:1081A0003F0210687B43090241431B1409140A2053
:1081B0008B4201DB584301E04843191CF7F7C8FF25
:1081C00056363378984208DD0123144923720E2075
:1081D000B62300220B71FEF7C9FC013D0E3C7AE785
:1081E000009F002F13D00B4B0E221B68019F1B6AB0
:1081F0005A43BA18013B0AD3111C0A390020095E00
:10820000002902DD911E012008700E3AF2E705B048
:10821000F0BDC046F8020020B40C0020BF030020CF
:1082200000030020F0B51C4B85B01B6803911B6A4E
:10823000DBB2013BDBB2FF2B2CD0039CD9006118D1
:1082400004254C5F9D005519002C1BD00E245C4367
:1082500004190427E65F002E14D02688019535B254
:10826000AC4600254F5F6546ED1B6F10BE19019FA0
:108270003E8064880225495F26B2711A49100C19A4
:108280007C80D6E70E21594341180C882C80498800
:108290006980CEE705B0F0BDF802002070B5124C41
:1082A000051C20680A226430002100F05BFF0F4BA0
:1082B00020681B681A6AD2B2013AD2B20023FF2AA0
:1082C0000AD00E21514369188B8081180E1C283664
:1082D000303133708B70EFE72268111C98319C327B
:1082E0000B60136070BDC04600030020F802002040
:1082F00070B50C4D002428680526031CA0331C60B3
:10830000321C211C823000F02DFF2868321C211CF9
:10831000873000F027FF2868211C0A226E3000F009
:1083200021FF70BD000300200F4AC378126810B50A
:1083300051685CB201398C4201DA0133C370837831
:1083400059B2002901DD013B83704378126859B2AC
:10835000013A914201DA0133437003785AB2002A9C
:1083600001DD013B037010BDF8020020F0B5B74DF0
:108370008BB007932B6805920C1C5A68B449049083
:1083800018684A709A68059E8A7001230132087045
:10839000CB70B218082306200B71FEF7E7FB2B68A1
:1083A000DB6ADBB2013BDBB2FF2B09D0049F1A0171
:1083B000BA187F2191721173FF21D1725173F1E7C5
:1083C000A44B00221B68119D1A600922AA56119D18
:1083D0000823EB569A4256DB119E0B217156119FD2
:1083E0000A23FB5699424CDB984B501C1E68B76819
:1083F000F66A7843059F013040183D182B78B34248
:1084000004DD3E2B3BD800232B7038E0002B36D008
:10841000109D4000405B8F4D013B2D682E6801365A
:108420002E60049EDDB22B01F318061C4E431F681C
:10843000BE191E60061C56435F68BE195E601E8929
:1084400086191E810C269E57B14200DA19730D263B
:108450009E57B14200DD59730A269E57B24200DA98
:108460009A720B269E57B24200DDDA72AD00651992
:108470000026AB5F834202DA2880EA70A9700139D6
:10848000ADE7013AA3E70026049F06966F4E069CCF
:108490003368DB6A9C4200DBE0E008203B5E002B97
:1084A00000D1DBE0381C0A300B24FFF73DFF3C57BE
:1084B00001940A23FB56019D9D4200DAC1E00D257F
:1084C0007D5703950C23FB56039E9E4200DAB5E0D0
:1084D0005E4B039C1E68019BB06801334343059DBE
:1084E00001331B19ED182A7800900295002A02D05A
:1084F0003F2A00D09FE0109D5B005C5B002C00D108
:1085000099E0002309930523013B002B24D0524A14
:108510000725D1180A1C4D5701214942515601988F
:10852000009A411801314A4305980399944642182C
:108530005219624451780029E6D0F26A9142E3DC94
:10854000002209A8855C002D01D18154DCE78D4211
:10855000FBD00132D2B2F4E709AA9A5CDDB2002A5C
:1085600004D00133042BF7D11D1C01E0002D62D093
:10857000291C201CF7F7ECFDF16A029E0131491914
:108580003170039E002246430096019E46430296A8
:108590006B1E9C4609AB9B5C049E013B1B01F318C0
:1085A000624513DA1E68241AB446009E0132B444B0
:1085B00066461E605E68B446029EB44466465E60CF
:1085C0001E89B446844466461E81E1E7039A186812
:1085D000624382181A60019A5E686243B2185A6058
:1085E0001A89A4181C810023122924DD634522DA8C
:1085F00001331A1CAA42F9DA09A8C118013909780D
:10860000105C01390138C9B2C0B20124814208D2DC
:10861000079E890071188440201C0C682043086064
:1086200007E0079E800030188C40211C046821431D
:1086300001600132DEE7039D013D42E7019C013C00
:1086400036E7069E1037013606961FE7F80200202F
:10865000B803002000030020309C00000025336890
:10866000DC6AA54205DA049F2C013C192789002FFA
:1086700016D1154A154912681868983215605A685B
:10868000059C4A709A6801238A7001320870CB7089
:10869000A2182D2306200B71FEF768FA0BB0F0BD6F
:1086A00021683FB20802391CF7F752FD626820606A
:1086B000391C1002F7F74CFD6060201C0A300135B0
:1086C000FFF732FEEDB2CAE700030020B803002036
:1086D000F0B54F4A4F4B12681B681179382251434D
:1086E00091B059182C31041C02A800F0F9FC4A4B37
:1086F00000211B685E681F680733DB7F013F013E76
:10870000FF1A36023F020191434D01992B681A6A04
:1087100091427BDA0421625E002A72DD3C4A1268D3
:108720001279012A6DD00022A05EFF2817DC0533E4
:10873000DB7F029903AA002B02D06B462A3301E0AB
:108740006B461633FEF7FBFA0021635E00B2013B75
:10875000FF3B584380110130FF30208019E0301A70
:10876000FF2816DC0533DB7F029903AA002B01D01A
:108770000DAB00E008ABFEF7E2FA0021625E00B24A
:10878000B21A013AFF3A5043731EFF3B80111B1A85
:1087900023800222A05EFF2817DC2B680299053394
:1087A000DB7F03AA002B01D008AB01E06B462A3324
:1087B000FEF7C5FA0221635E00B2013BFF3B58435E
:1087C00080110130FF3060801BE0381AFF2818DC70
:1087D0002B6802990533DB7F03AA002B02D06B467E
:1087E000163300E00DABFEF7AAFA0221625E00B27A
:1087F000BA1A013AFF3A50437B1EFF3B80111B1A05
:108800006380019A0E34013201927DE711B0F0BD10
:1088100000030020B80C0020F8020020F8B5144E28
:10882000041C33680D1C0633DF7FFEF7F3F9114B90
:108830001B68E6331B781840336878405A1DD27F96
:10884000002A0BD02288298821802A8000280DD078
:108850001A680733DB7F013AD31A03E0002805D0FA
:108860005B68013B22881B029B1A2380F8BDC0462F
:10887000F802002000000020F0B5038889B007ACA2
:1088800002902380438869461E31201C0B80FFF72D
:10889000C5FF334B1B685A1DD17FDD1D314A81CB8B
:1088A00000290CD01268EB7F411E013F9068C91A65
:1088B0003F02DB01049709021B18D7680BE0791E01
:1088C0001268EF7F0138C01B9368D2680002FF0175
:1088D00009020490BF18244A6D4616681E35326896
:1088E00001920022A05E019AC0185B00C918504393
:1088F000F7F72EFC80B2059020807068049B0390EF
:108900000021685E039AC0197F00D9195043F7F718
:108910001FFC331C80B22880059FD4331B783AB2E9
:108920009A4206DD019FF91A8A4203DB3A1C013A9A
:10893000D31A2380D536337800B2984206DD039FE0
:10894000FA1A904203DB3A1C013AD31A2B8007AB88
:108950001B88029F01333B802B887B8009B0F0BDD0
:10896000F802002000030020B80C0020024B1B6816
:10897000983318687047C0460003002038B5041CBF
:10898000081C002A07D0D118584362434D10101814
:108990004019F7F7DDFB38BD10B5F7F7A3FD054B20
:1089A00001781C68044BFC341B68D868F7F782FB1D
:1089B000606610BD00030020B40C0020F0B56A4BC7
:1089C0000C1C1B6809791B68071C151CFA206279AE
:1089D00085B0800000915043191C02930392F7F771
:1089E000B7FB624B1B6898331B68002B18DD012610
:1089F000012B18D15E4B1B681A6A013A0ED30E2365
:108A00005343FB1804215B5E002BF6DD5949012618
:108A10000968E03109888B4207DB04E0012604E0A5
:108A20000026012200E0321C52420E235343FF185D
:108A30003B8801937F88022D17D004D8002D0AD0DF
:108A4000012D0DD088E0052D30D0062D50D0042DFD
:108A500000D081E027E0002A60DA012E2ED17DE0EF
:108A6000002A62DA012E6ED178E0002A03DB009939
:108A70004F295AD972E0009AFA2080005043029997
:108A8000F7F766FB3B4B1A68131CE2331988032384
:108A9000884205DCE43212880023904200DA052384
:108AA000012E35D15AE0012E08D159E0002E07D110
:108AB000304B1B68E4331B88984244DB082350E0AA
:108AC000002AFBDB0199236808B200215A5E3FB2FD
:108AD000801A02229B5EF91AFFF7B4F8254B1B6837
:108AE000DE331B789842E9DC00236371062338E00B
:108AF0000723002E35D00423002A32DB1D4A1268DA
:108B0000E432128890422CDA63790133637127E0F2
:108B1000022B0AD0052B16D0012B22D123680199F4
:108B20005F801980012323711BE0009923688A006C
:108B30000199D152227992009B185F8023790133E9
:108B4000237102230DE0013D0023012D01D9039B78
:108B500001336371052304E0002302E0042300E0F5
:108B60002B1C181C05B0F0BD0000002000030020E5
:108B7000F8020020B80C0020F7B5141C0422061CD3
:108B80000D1C019300F0ACFA0198324A371C811891
:108B9000890070180422691800F0A2FA01230093DA
:108BA000019B0098013B0435043798421CDA2B1FC7
:108BB0000022985E0022AB5E0321C0180422AB5E47
:108BC000C018F7F7C5FAAB1E38800022985E022263
:108BD000AB5E0321C0180622AB5EC018F7F7B8FAE7
:108BE000009B78800133DAE773880025E380A38057
:108BF0003388012763802380019A974227DA002275
:108C0000B35E0422B05EC01A0623F15E0222B35E98
:108C1000C91AFEF7F1FFB3882D180220215E1AB29F
:108C2000914200DA63800020215E914200DD2380C2
:108C3000F3880622A15E1AB2914200DAE380042092
:108C4000215E914200DDA38001370436D4E7281C61
:108C5000FEBDC046FFFFFF3FF0B58BB0059003910E
:108C6000101C14210893F7F773FA01240690039956
:108C70000598042200F034FA00270194019B08991A
:108C80008B4246DA0199039A8B000399D218043B70
:108C90000292CD1800216B5E0020105E029AC01A6D
:108CA0000221515E0222AB5EC91AFEF7A5FF0699AA
:108CB0003B1804908B4227DB0023EA5ECF1B079210
:108CC000029A02216E5E0220105E0499801B784396
:108CD000F7F73EFA029930180990079A0020085ECB
:108CE000059B801AA600049978439E19F7F730FA7D
:108CF000079B0999181880B28BB2738030800134B9
:108D00006B802880002302E0019A013201921F1C2F
:108D1000B4E7142C0AD1064BCA18039992008A189A
:108D2000059B11885033198052885A800BB0F0BDD2
:108D3000FFFFFF3FF7B5051C04228B5E0622885E0D
:108D40000C1CC01A642358430223C95E0022A35E90
:108D50000026C91AF7F7FCF9371C01900222AB5E16
:108D6000642001995843F7F7F3F981B26980012F24
:108D70000DDD0023E85E2B1F00229B5E09B2C01AA6
:108D8000AB1E00229B5EC91AFEF736FF361801376C
:108D90000435152FE2D10423E05E64256843019970
:108DA000F7F7D6F9A0800622A05E01996843F7F78D
:108DB000CFF9E080301CFEBDF0B593B001900F1CE0
:108DC0000D1C0026142E0BD13B1C4C330020195EC9
:108DD00000203A5E8A1A0220195E02203B5E08E0FB
:108DE00000202B5E04216A5ED21A0623E95E02206F
:108DF0002B5ECB1AA821FF315143012489128B42EB
:108E000000DC0024184842439212934201DD022004
:108E100004435242934201DA0422144349428B42F2
:108E200001DA08231C430021402202A800F09AF92D
:108E3000012302930223039303230593042309933D
:108E400008230A9307230E9306231093A4000523F7
:108E50001193083469466358019A043593550136D5
:108E6000152EAFD113B0F0BDA7090000FFB5051C4A
:108E7000FFB0002601242B799C4213DA2B68A10055
:108E80005A1804395B180021505E0027D95F01345D
:108E9000401A0227D15F02229B5EC91AFEF7D2FE5A
:108EA0003618E8E7194A00241268DC321288964224
:108EB00027DD296801AA32A8FFF75EFE2B79021C84
:108EC00032A91DA8FFF7C8FE6B4603A81DA9DC70D8
:108ED000FFF772FF6846033003A9FBF7AFFA6F464E
:108EE000FB78041C002B0CD101A91DA8FFF722FF61
:108EF0001DA9021C09A8FBF75BFA09A8FBF7DEF91C
:108F0000041C201C83239B009D44F0BDB80C002052
:108F1000014B18607047C046BC0C0020014B18681C
:108F20007047C046040300200048704764060000F4
:108F3000024B1868DD30FF307047C0460403002044
:108F4000A2235B005843A6239B00C018014B1B685B
:108F50001818704704030020DF235B005843014BBF
:108F6000C018704774BA00000A2358439E239B0020
:108F7000C018024B1B6818187047C0460403002035
:108F800008B5FBF789FA0E4B41791B6859604279A5
:108F900002329A6082791A604A43DA604279022189
:108FA0009A615200DA61026859611A62C2791A61E3
:108FB00001795A1DD17702790633DA7708BDC046A8
:108FC000F802002010B5134C1349144A206800F031
:108FD00087F82068FBF75AFA20687C30F7F770FAB8
:108FE0002068B830FDF7C4FE2068C030FEF7CAF92B
:108FF0002068D930FF30FDF773FBFFF7C1FF084C45
:10900000201CFBF75BFADF239B00E018FDF7C8FE8E
:1090100010BDC0460403002010B400006406000028
:1090200074BA000038B5164BA224596864000A7857
:109030001B685443A6229200A4181C19114B201C33
:109040001C60FBF72FFA98235B00E518281CFFF73C
:109050005FFF201C9C30F7F73FFA201CB430FDF76F
:1090600093FE201CC830FEF799F9281CFDF73EFB43
:10907000054B5A341B6822780733DA7738BDC0466F
:1090800004030020C00C0020F8020020014B5B68A4
:109090001870704704030020014B5B681878704714
:1090A00004030020F8B50D1C041C081C111C161C20
:1090B000F7F74EF8311C071C281CF7F79FF8002D16
:1090C00005DB002908DB2760201C6160F8BD002952
:1090D000F9DD013F8919F6E70137891BF3E7C0463F
:1090E000F0B50F2A35D9031C0B439C0735D1161C4C
:1090F000103E36093501451910350C1C031C276834
:109100001F6067685F60A7689F60E7681034DF6072
:109110001033AB42F3D1731C1B01C518C9180F23C0
:109120001340032B1BD91C1FA4080134A4000023E7
:10913000CE58EE500433A342FAD1ED18C9180323D8
:109140001A4005D00023CC5CEC5401339342FAD191
:10915000F0BD051C002AF5D1FAE7051CF2E71A1C40
:10916000F8E7C046F0B5830746D0541E002A42D027
:10917000CEB2031C032503E0621E002C3BD0141C5E
:1091800001335A1E16702B42F6D1032C2BD9FF2522
:109190000D402A0215432A0415430F2C15D9271C0C
:1091A000103F3F091E1C3A011036B6181A1C1560F4
:1091B00055609560D5601032B242F8D101373F0159
:1091C0000F22DB191440032C0DD9271FBF08BA004A
:1091D0001E1DB6181A1C20C2B242FCD10137BF00B6
:1091E0000322DB191440002C05D01C19C9B21970D8
:1091F0000133A342FBD1F0BD141C031CC5E7C046DC
:109200000405AE0174033B050207CD08940A590C0E
:109210001F0EC7FD8FFB4FFE1DFC70F8230199FC4C
:109220003EFED1FC30FCF0FD7DFFDAFA66FCD7FC97
:10923000AFFBCDFD83FA5DFD7AFF04FD8BFD67FD7D
:10924000B1F8030254FF2BFFFCFFC5FF8E006CFF3B
:1092500081FF29FF8EFF4CFFB7FF78FE5DFFE1FE27
:1092600001FF3100C4FFDA003A009900C80029016B
:10927000B800230166008D0030FF6B007BFE030009
:10928000DFFE31003FFE3E005AFED7FFEEFEF3FE4A
:109290008600F6FF14010000A900A7FF50009DFF03
:1092A0009B004DFF310002FF27000B005A006FFFAB
:1092B0002800DFFE900025FF9EFF9AFFE2FEF3FFED
:1092C000ECFE290065FFB000FBFF0F01F7FF140162
:1092D000F7FFB60051FF780041FFC6FF20FF2A00CC
:1092E000E4FE1700D1FFFBFF6CFF6D0085FF4A0015
:1092F000FCFF6901A600BD006600C4FF11008F00DD
:10930000D0002A00EAFF44FF64FF52FFE0FF92FF13
:109310002C000B000301D8FFA4009A00CC00A80089
:109320006B00A80072001F014B01F900B401260078
:109330008400F4FF49FF8CFF87FF82FFD7FFE0FF27
:10934000D0FF59FF74006700500017011D00A700EF
:109350000B00BF00BAFF4400BCFFB7FF12009CFF28
:109360004000EFFF1100730085FFBB00AAFF06005D
:10937000A5FF16FF63FFDCFEADFF21FFDCFF8A01C6
:10938000E5FEE201FEFF0B000301F9FF7D01CFFFC7
:109390000A01ABFFA50027FFF9FFE7FE07005CFF0E
:1093A00002FF1700B1FE280079FF99001900F0FFB5
:1093B000ECFFEFFF53001B00C7005D0011016201CD
:1093C000E9008A007501ACFF48012AFF5C00E4FF58
:1093D000720015FF70000100DAFFB1FFBE00DFFF71
:1093E00031007BFFF6FF3600CE0047007900B9FF61
:1093F0007000CFFF3A005EFF4000AAFF100096FF0A
:10940000BCFFEFFF5100F7FF790177FFCF0153FF5A
:10941000420109007300940079009E01C300E3013A
:10942000F0FF62016300DEFFAB011300B801010031
:10943000B7007300E8FFD80081FF000181FF3A0107
:1094400032FF310110FFB500E2FF13009FFF9CFFC8
:10945000D8FF200099004200EBFF6C00B6FF4B00E4
:10946000EBFFDFFF0F00EEFFDCFF54002D00D40008
:109470000A001400D6FF5EFE7CFF76FEA0FFA6FE6B
:10948000E3FF36FFFAFF8600B3FFC50040FF15007B
:109490005FFF6EFFCCFFF8FEF1FF06FF1A00A2FF90
:1094A0003300ECFF0C003E0084FF6100DEFF420051
:1094B0006900DAFF5E0058008D00EF0049001600D9
:1094C000F4FE4700A00041FFA300960045003901CB
:1094D000E7FF0001F6FF4D00E4FF27007900AAFE38
:1094E000040196FEE600F3FF930099FF4C00630031
:1094F000DBFFAB016C00A4003800F6FFDA0028FFA8
:109500004B0024FF160035FFF9FF35FF32FF6FFFD8
:10951000C8FF2700BEFF69FFFFFFEEFED3FE08FF76
:10952000B9FE80FF9EFE6EFE30FFD0FE4000B8FE0A
:109530002B008EFE0C00FBFEC3FF5DFF29FFC3FE68
:1095400054FF1CFFC6FF3DFFBCFF7100D2FF7B0034
:109550003D0072FFF4FFE7FE0CFFA5FE65FF7FFFF5
:1095600013006D004A001C0079FF99FE20FF36FFB2
:1095700049FFC1FF0E00DEFF470013FF7AFF27FF00
:1095800074FFCAFF26FF7400B2FF98004C00CD00A4
:1095900088007A007800BF0089008F00F4FFD7FFB1
:1095A000F0FF96FF350024006A006B0071003C005C
:1095B000B100B8FF0E008DFF4D005B006700010099
:1095C000030086FFBBFFDFFEFEFFE3FEBAFFF4FEF3
:1095D000B6FFD5FF050040011E00D8002A00390063
:1095E0002800F0FF67005AFF0E0011FFE6FF9BFF07
:1095F000CFFFF0FFE1FF6300D9FF7600C5FF510008
:10960000C2FF5000F6FF7D00DDFF65FF1200EEFF98
:10961000E8FFDDFFA8FFD8FF820063003000A20052
:1096200092FF5A00ADFF7B00FEFF0600E5FF3C0005
:1096300094FF8B00F9FE610021FF64006EFF55FF6F
:1096400030009BFE1A00A0FEC7004500DD014B0064
:109650006802DAFF20FF5A00A4FFFAFF81FFD6FF5D
:10966000EAFF8D00B4FF84006DFFBB0076FF580059
:10967000D7FF95FFD9FF50FF5B00BEFFE5FF27FF37
:109680006500EFFE1B00C4FEBFFFDDFE38FF9AFF42
:10969000EEFE3F0048FF1000AFFF6800EAFF6800E1
:1096A0000301B7002C00E1FF5800AAFFA2009EFFB3
:1096B000AB005200E70086008A006D005F016D007C
:1096C000B8006C00B5FFFC00BEFF1B011400D50004
:1096D0001500E00091FF920038FFEFFFCEFFF1FF91
:1096E0005D00A4FF2700F1FFE4FFA3FF4E00BAFFD7
:1096F0003BFF730041014600D700E400BB001E00A1
:10970000F0000A006E005F008200CA00C0007E0107
:109710008500F500B900C8FF65007200D000C0FFE9
:10972000F900B9FEA10067FEC20003FFB8003100D6
:1097300083009A004A0092FF7B0026FF7A00CFFE4A
:109740007200360043FF4DFF1AFFDEFE64FFE7FEA6
:10975000C3FF41FFA2FFF7FE430045FF300159FF61
:10976000FB005DFF4F0067000900BE0017FFBF0050
:1097700063FFB0FF7500C6FEA20040FFB4004D00BD
:10978000D1FFD8000300AB00EBFFCEFF040052FF77
:1097900045005BFF40FF3C00E2FEC1FF1EFE65FF8F
:1097A0005EFEEFFE21FFEFFFF0FF9900F1FFBE002C
:1097B000C9FF14016200A3015A00B901B900FB00FE
:1097C000BF002001C4FF06021F00F00142FF6E002F
:1097D000E3FF3400A9FFE8FFE4FFA9FFC6FFE5FFB0
:1097E0006F00E0FF8AFFD2FFE1FFC2FF170053FFC7
:1097F000F2FFDAFFCFFFBDFF4EFF300033FF57000F
:1098000018FFF4FFAFFE58FF39FF10FF3CFFCFFEFB
:109810008CFF86FE4DFF62FEF3FEC6FEAEFE5BFFD2
:10982000F2FE4D0039005A003A0112000901E4FF2E
:10983000BE009B00B8FF4000890089010900DE00DE
:10984000FDFF4D00D5FF3300ADFFA6FF7DFEEBFF12
:109850009AFF23001B0010FFD00055FF67015F0037
:109860001401390095FFC3FFC3FE4100FCFFA300B4
:109870003600A600E3FF8800A200D500940027016F
:1098800019FFB600BDFF4700F5FF8F005E003F00E7
:1098900006008BFF6000DBFF6A006BFFBA0070FF01
:1098A0002F0000FF85FF3D008AFF460051FF550055
:1098B000C5FFB8FFDCFF78FF8BFFAFFF63FF25001C
:1098C00092FFF900870018018600CD000200F00029
:1098D0005AFF46018B0098FFB3FFCE01E6FF5E0101
:1098E000910099002E0001004000640073002C00DC
:1098F000FAFF75FFA1FF14005EFF2C00DFFEDB0006
:10990000EBFFF7FFDA008F00A200D5009CFFF6FF07
:10991000F8FE59FF11FF3FFF27FF5CFF97FF06FF8F
:1099200095FF87FFB4FFBFFF52FF21FFA2FFE3FFB8
:10993000B8FF4700E5FF3300D3FFF3FF3FFF2A00E6
:1099400058FF4200B6FF5B0098FF4F0050FFF5FF45
:1099500029FF0B00C9FFA5FF31001CFF5000A2FE2C
:10996000F9FFC3FEA3FF8AFFEDFEE0FF90FE250096
:1099700099FE8BFF49FFF00095FD8E0027FEAA009F
:10998000B5FE81001EFF98000D004C000201320060
:109990005B013000EA016100A800D8003000C70078
:1099A000B1014F0031012400D900E8FF63FF95FFAA
:1099B0003FFF6DFF9CFE96FF5EFEF5FFE4FD0AFF94
:1099C0006DFF650009FF82FF84FF4500C3FFA9FF0B
:1099D000470079006900EB0083003F015500CF008C
:1099E000D2FFDF007EFF9001F9FF160179FF5000E2
:1099F0004EFF210027002400090047014300BE005C
:109A00008200DF0058003F011D0022013D007B0065
:109A100073FFC4FFE800F500D402B5046FFF3AFC01
:109A2000D0FD46FDDCFF0C027902E4027FFD60FD03
:109A30009901BDFF9200E4FE9F03E10188001A0333
:109A40006C016AFF1002F1003AFD3E00AC0290FD8D
:109A50006402F00079010E01E5FC90FF9CFFCCFF51
:109A60007E00F1FD0700F300B0FFCCFE3D01A4FE37
:109A7000F7FE87FF2BFFD4FF1CFE3F0222FFF8FEFC
:109A8000C2FFDEFF02FFC0008C01A9FFB1FFC6FFCD
:109A9000D2FF41FF24FFACFFE9FFE7020D0073FF97
:109AA000B60144FFD0FF62FFEFFE43FF6CFF6F0083
:109AB00022FE9BFF9201E8FF31FFA2FFD2FF93FF3E
:109AC0005FFE6100C0FFAAFF77FDBEFFF9FEEEFF5B
:109AD000B7FFFAFEA1FE2AFFBE015B0386FF3FFF30
:109AE0005AFDA9FFC9FF3BFF70FFC1FBDBFD56FF1D
:109AF000C5FEE9FF90016DFF6202DDFF9602A40141
:109B0000C8FFA0FE0201D7FF9AFE6FFFF4FE2902F4
:109B1000E5FEB3FE4D016700B6FFE0FE12FFB3FFA6
:109B2000B40243FF1400010114017301FEFF6BFF37
:109B30005AFFB0FFE5FE3E00B4002DFF0B0097FF7B
:109B40009EFE5201FA01BEFF8700ABFE8FFF0802A6
:109B500013009FFFFAFEA4FFDFFFDE00E9FF9A0279
:109B600088FEEFFFA9000DFF15FFECFFEEFF2102BD
:109B70003EFFDA01520091FFD5FF90006BFFC7FF57
:109B8000C3FF510291FF480194FF2F0096FF75FE1D
:109B900063002E0071FE74FF3D0045FFF0FF670279
:109BA000E6FF11FE2DFFC100C00248FFD20047FFB3
:109BB000CD0215024DFE5D006B002700E3FF2C0275
:109BC00078FF40001EFE2F0006FEEB008900A6FF76
:109BD000F9FFCBFEFAFF5D009300D8FF6B00FA009F
:109BE000E0FFB4FFE4FF84FF31FF1FFE5CFFFC03D6
:109BF000A6FFCE059500B506A8017E062E02010639
:109C00001F025C056A02B50477031D048704710313
:109C10000C0521032705EA02700549022F06FD0104
:109C2000A406D601AA068A016106B60157062001DC
:109C30004D07BAFF4E0855FEC30B510DAD0DA90ED1
:109C4000440D980E820C610EE90B4E0EA70B290EE7
:109C5000CC0B790EE50BBC0EF40BA50E140C550EB7
:109C6000D50BED0E950B510F870B310FB50BB50EC4
:109C7000810C280E050DCB0DD30D800DEB0E560D6E
:109C8000F90E180D7B0BBA0A060000000800000050
:109C9000FF000001FF01FF0100FF0100FFFF0101C4
:109CA00000010203040405060708090A0B0B0C0D4A
:109CB0000E0F101111121314151516171818191A62
:109CC0001B1B1C1D1D1E1F1F20212122232324249A
:109CD0002525262727282829292A2A2B2B2C2C2DF5
:109CE0002D0000007804EF08660DDB115016C21A33
:109CF000331FA1230C28742CD93039359639EE3D09
:109D000042429046D94A1B4F58538E57BE5BE65F7E
:109D100007641F68306C397038742F781C7CFF7FA3
:109D2000D983A8876D8B278FD5927996109A9B9DA2
:109D30001BA18DA4F3A74BAB97AED4B104B526B845
:109D400039BB3EBE34C11BC4F2C6BAC973CC1BCFEB
:109D5000B3D13BD4B2D619D96EDBB3DDE6DF08E26E
:109D600018E416E603E8DDE9A5EB5BEDFEEE8FF007
:109D70000DF277F3CFF414F646F764F86FF967FA4B
:109D80004BFB1BFCD8FC81FD17FE98FE06FF5FFF16
:109D9000A5FFD7FFF5FFFFFF040000200000000033
:109DA000FF000000000000000000000000000000B4
:109DB00000000000000000000000000000000000A3
:109DC0000000000000000000000000000000000093
:109DD0000000000000000000000000000000000083
:109DE0000000000000000000000000000000000073
:109DF0000000000000000000000000000000000063
:109E00000000000000000000000000000000000052
:109E10000000000000000000020000000000000040
:109E20000000000000000000000000000000000032
:109E30000000000000000000000000000000000022
:109E40000000000000000000000000000000000012
:109E50000000000000000000000000000000000002
:109E600000000000000000000000000003000000EF
:109E700000000000000000000000000000000000E2
:109E800000000000000000000000000000000000D2
:109E90000000000020030020C60300200100000095
:109EA00000000001030084000000000053040020B3
:109EB000000000000000000047040020EB0200202A
:109EC000DF020020DD020020CC020020C8030020B9
:109ED000D6010020D803002002000000400400202A
:109EE0003F040020EA03002007000000E8030020F0
:109EF000BB020020B902002000000000B1020020D7
:109F0000E903002000000000000000000000000045
:109F1000000000008C0200207802002000000000F9
:109F200000000000000000006402002000000000AB
:109F30005002002000000000380200200000000055
:109F40001C020020000000000000000000000000D3
:109F500004020020F0010020DC010020AD020020FE
:109F6000A802002000000000E30300200001002000
:109F700000600000D0010020E0030020EC01002080
:109F8000010000000500000054010020E103002052
:109F9000000200200100000001000000C4010020B8
:109FA000170200201402002003000000040507002F
:109FB0001020000064010020310200202C0200204B
:109FC00005000000080106010400102030310000E7
:109FD000580100204B02002048020020030000002E
:109FE0000802060010200000C4020020E203002046
:109FF0006002002001000000040000002C0100208D
:10A0000076020020740200200200000002110010FD
:10A0100044010020880200205001002003000000BD
:10A020000010110014010020A20200209C02002058
:10A03000060000001708080C0A0C00203040507081
:10A04000010000000000200601002001021E0001A6
:10A0500000FF00002001027E00000000C802002076
:10A060000060090100010000000000000000000085
:10A0700000000000000500004D3448304D45000050
:10A080000000004D495000000000000004000000E6
:10A0900070040020A0040020B00400201806002056
:10A0A00014060020FFFFFFFFFFFFFFFFFFFFFFFF82
:10A0B000FFFFFFFFFFFFFFFFFFFFFFFFFFFFFFFFB0
:10A0C000FFFFFFFFFFFFFFFFFFFFFFFFFFFFFFFFA0
:10A0D000FFFFFFFFFFFFFFFFFFFFFFFFFFFFFFFF90
:10A0E000FFFFFFFFFFFFFFFFFFFFFFFFFFFFFFFF80
:10B45000FFFFFFFFFFFFFFFFFFFFFFFFFFFF0501F4
:10B460004D3448305041524130303030303030303F
:10B470000A00000001180E000100000B0A0908076D
:10B48000060504030201001A1B1C1D1E1F20212299
:10B49000232425191817161514131211100F0E0D49
:10B4A0000C00000000000000000000000000000090
:10B4B00000000000003F1D06BF00F000000000007B
:10B4C000000000000000000000000000000000007C
:10B4D0000000000F000000000000000083000000DA
:10B4E0000001E1A108000009030300004E45574A8E
:10B4F000375F464844000000000000000A32320076
:10B500000100FFFFFFFFFFFFFFFFFFFF0A05F40140
:10B5100008072D005A001E000005641E1E14100F9F
:10B520003C000000000000000A0A32000080000019
:10B530003804000080070000C8000000200300005D
:10B54000C8000000E80300006400000001000000E3
:10B5500001000000010000000100000005000000E3
:10B56000000040008000C400FF005E0054004C005A
:10B57000460040005E0054004C00460040005E0063
:10B5800054004C00460040005E0054004C00460051
:10B59000400000000000000000000000000000006B
:10B5A000000000000000000000000000000000009B
:10B5B000000000000000000000000000000000008B
:10B5C0000000000000000000000000000200000079
:10B5D000000040008000C400FF00800080000000E8
:10B5E00000000000800080000000000000008000DB
:10B5F00080000000000000008000800000000000CB
:10B60000000000000101A802BA043C00C8001E00AE
:10B61000B0045E01F4014B0090010100080000003D
:10B62000000018003F00610080009F00C500FA0084
:10B63000000000003C002B0020001D001B00190032
:10B640001700140000000000010000003200F000AC
:10B6500000000000000000000000000000000000EA
:10B66000000000000000000F0000000000000000CB
:10B670001E00F000000000000000000000000000BC
:10B6800000000000000000000000000F00000000AB
:10B69000000000008000000040033318D10000715A
:10B6A0000A48F61C000000320F05320F00320F0569
:10B6B000000000000000000000000000000000008A
:10B6C000000000000000000000000000000000007A
:10B6D000000000000000000000000000000000006A
:10B6E00000000000000000000000FFFF0A143807FF
:10B6F00003000000FFFF0A14380703000000FFFFEB
:10B700000A14380703000000B200F0000000000037
:10B710000000000000000000000000000000000029
:10B720000000000F00000000000000009E00F0007C
:10B730000000000000000000000000000000000009
:10B74000000000000000000F0000000000000000EA
:10B750008000000040033318D10000710A48F61C35
:10B76000000000320F05320F00320F05000000000C
:10B7700000000000000000000000000000000000C9
:10B7800000000000000000000000000000000000B9
:10B7900000000000000000000000000000000000A9
:10B7A000000000005A1EFFFF0A0000000700000012
:10B7B000FF7F0080FF7F0080D8FF00000103470269
:10B7C00000005A030A0000800A070A0A0CF9400028
:10B7D000B003520326025E01300000001027000073
:10B7E0000800000000000C000D000E000F001E00FD
:10B7F000320046003C003C003F00460051005A0029
:10B80000820082004B820000E10000001E0F020156
:10B81000020200000F0000000F00000001011400F0
:10B820000000DC0578001900FA000613133D8002C1
:10B83000000120006000000001000A0D1E003C0015
:10B840000810081000002C01E8031000B200F000FE
:10B8500000000000000000000000000000000000E8
:10B86000000000000000000F0000000000000000C9
:10B870009E00F0000000000000000000000000003A
:10B8800000000000000000000000000F00000000A9
:10B89000000000008000000040033318D100007158
:10B8A0000A48F61C0000003F1D063F1D003F1D0614
:10B8B0000000000000000000000000000000000088
:10B8C0000000000000000000000000000000000078
:10B8D0000000000000000000000000000000000068
:10B8E00000000000000000005A1EFFFF0A000000D8
:10B8F00007000000FF7F0080FF7F0080D8FF00006E
:10B9000001034C0200005A030A0000800A070F0AD4
:10B910000CF940004C03EE02C201FA0030000000B6
:10B9200010270000080000000000070009000A00BE
:10B930002100270046005A00320032003200320057
:10B940003200BE00DC00DC005A8C0000DC0000008D
:10B950001E0F020102020000070000000F0000009D
:10B96000010114000000080769001900FA00061917
:10B97000133D800200012A00800000000100060D36
:10B9800028005A001428142800002C01E803100095
:10B99000BF00F000000000000000000000000000F8
:10B9A00000000000000000000000000D000000008A
:10B9B000000000009E00F0000000000000000000F9
:10B9C0000000000000000000000000000000000F68
:10B9D00000000000000000004000000040033B1891
:10B9E000D10000710A48F61F000001380F053F1D05
:10B9F00000230F0500000000000000000000000010
:10BA00000000000000000000000000000000000036
:10BA10000000000000000000000000000000000026
:10BA2000000000000000000000000000781EFFFF82
:10BA30001400000007000000FF7F0080FF7F0080EF
:10BA4000D8FF00000003000000005A030800008037
:10BA500007070F0A0FF64000B003520326025E01EB
:10BA600030000000102700000700000015002B0028
:10BA70002C0034003A0056006E0000003C006400C8
:10BA8000CF00CF0090010502050200004BA000008E
:10BA9000900100001E0F02010202000007000000DA
:10BAA0000F000000010114010000080769001900DF
:10BAB000FA000619133D800200012A0080000000F0
:10BAC00001000A0D2C01E8030F3C0F3C00002C0183
:10BAD000E8031000080809090A0A0A0A0B0B0C0CF3
:10BAE0000D0C0D0D0D0D0D0D0D0D0C0E0808090999
:10BAF0000A0A0A0A0B0B0C0B0D0D0D0D0D0D0D0D89
:10BB00000D0D0D0D080809090A0A0A0A0B0B0C0B8A
:10BB10000D0D0D0D0D0C0D0D0D0D0C0D080808096A
:10BB2000090A0A0A0A0B0B0C0C0D0C0D0D0C0D0D5D
:10BB30000C0D0D0C0708080909090A0A0B0B0B0B61
:10BB40000C0D0D0C0D0D0C0D0D0C0D0D070708083F
:10BB50000909090A0A0A0B0B0C0C0C0C0C0C0C0C36
:10BB60000C0C0C0D07070808090909090A0A0B0B38
:10BB70000C0C0B0C0C0B0C0C0C0C0B0D060707081B
:10BB800008090909090A0A0B0B0B0B0B0C0B0B0C10
:10BB90000B0B0C0B0607070808080809090A0A0A14
:10BBA0000B0B0B0B0B0B0B0C0B0B0B0B06060707F6
:10BBB00008080808090909090A0A0A0B0B0B0B0BEC
:10BBC0000B0B0A0B060606070708080808090909EF
:10BBD0000A0A0A0B0B0A0B0B0B0B0B0B05060607CD
:10BBE00007070708080909090A09090A0B0B0A0BC4
:10BBF0000B0A0B0B050506060707070708080809C7
:10BC00000909090A0A0A0A0A0A0A090B05050506AA
:10BC100006070707070808090909090A0A090A0A9D
:10BC2000090A0A09000000000000000000000000EE
:10BC30000000000000000000000000000000000004
:10BC400000000000000000000000000000000000F4
:10BC500000000000000000000000000000000000E4
:10BC600000000000000000000000000000000000D4
:10BC700000000000000000000000000000000000C4
:10BC800000000000000000000000000000000000B4
:10BC90000000080809090A0A0A0A0B0B0C0C0D0C13
:10BCA0000D0D0D0D0D0D0D0D0C0E080809090A0ADC
:10BCB0000A0A0B0B0C0B0D0D0D0D0D0D0D0D0D0DC1
:10BCC0000D0D080809090A0A0A0A0B0B0C0B0D0DC9
:10BCD0000D0D0D0C0D0D0D0D0C0D08080809090AB0
:10BCE0000A0A0A0B0B0C0C0D0C0D0D0C0D0D0C0D96
:10BCF0000D0C0708080909090A0A0B0B0B0B0C0DA0
:10BD00000D0C0D0D0C0D0D0C0D0D07070808090984
:10BD1000090A0A0A0B0B0C0C0C0C0C0C0C0C0C0C6E
:10BD20000C0D07070808090909090A0A0B0B0C0C76
:10BD30000B0C0C0B0C0C0C0C0B0D06070708080960
:10BD40000909090A0A0B0B0B0B0B0C0B0B0C0B0B49
:10BD50000C0B0607070808080809090A0A0A0B0B52
:10BD60000B0B0B0B0B0C0B0B0B0B0606070708083A
:10BD70000808090909090A0A0A0B0B0B0B0B0B0B24
:10BD80000A0B0606060707080808080909090A0A2F
:10BD90000A0B0B0A0B0B0B0B0B0B05060607070711
:10BDA0000708080909090A09090A0B0B0A0B0B0AFB
:10BDB0000B0B050506060707070708080809090908
:10BDC000090A0A0A0A0A0A0A090B050505060607EE
:10BDD0000707070808090909090A0A090A0A090AD6
:10BDE0000A09000000000000000000000000000040
:10BDF0000000000000000000000000000000000043
:10BE00000000000000000000000000000000000032
:10BE10000000000000000000000000000000000022
:10BE20000000000000000000000000000000000012
:10BE30000000000000000000000000000000000002
:10BE400000000000000000000000000000000000F2
:10BE5000242527292A2C2D2E3031333434363536FB
:10BE6000363738373738393F2221232425272829E8
:10BE70002A2B2C2E2D2E2F2F3031323232323239C6
:10BE80002221232425272728292B2B2D2C2E2E2F2A
:10BE900030303131313132382220232425262628F2
:10BEA000292B2B2C2C2E2E2F2F30303131313238A4
:10BEB0002221232425272728282A2B2B2C2D2E2FFF
:10BEC0002F303031323132392221232425262728C0
:10BED000282A2A2B2B2C2D2E2F2F30303130313980
:10BEE0002321232425262728282A2A2B2B2C2D2ED4
:10BEF0002E2F303131313139222122242526272796
:10BF000028292A2A2B2C2C2D2D2F2F303030313858
:10BF1000222021242526262828292A2A2B2B2C2CAE
:10BF20002E2E2F2F30303037212021222425262776
:10BF30002729292A2A2B2B2C2D2E2E2E302F303537
:10BF4000211F212224252626272829292A2B2B2C8C
:10BF50002C2C2D2E2E2E2F341F1F2021232425265E
:10BF600027282929292A2B2B2B2C2D2D2D2E2E321B
:10BF70001E1D1F222324252626282929292A2A2A6C
:10BF80002C2C2C2D2D2D2E322121232627292A2B16
:10BF90002C2E2E2F30303131323233333231313496
:10BFA0000000000000000000000000000000000091
:10BFB0000000000000000000000000000000000081
:10BFC0000000000000000000000000000000000071
:10BFD0000000000000000000000000000000000061
:10BFE0000000000000000000000000000000000051
:10BFF0000000000000000000000000000000000041
:10C000000000000000000000000000000000FFFF32
:10C01000FFFFFFFFFFFFFFFFFFFFFFFFFFFF050128
:10C020004D4254014D3448300000000000C0000073
:10C03000EEEE050205010501EEEEEEEE002D2D30CF
:10C0400000220901000C00000801162024412200F2
:10C050000000000000000000000040001BF800008D
:00000001FF
